:020000041100E9
:103000007FB50023284C294D03932800217C284AB2
:1030100001F0CDFA002812D103232800217C03AA55
:1030200001F06CFA00280AD1224B039A9A4206D189
:10303000214B2248E360224B636104B070BD02263D
:10304000217CFE2228001F4B009601F029FA00285F
:1030500001D00020F1E71C4BA2899A42F9D1217CD2
:10306000FF222800194B009601F01AFA0028F0D12F
:10307000E389174A934203D1164B17486361DCE793
:10308000164A9342E5D1164B164A1B68934206D95D
:10309000C02304222800217C9B0001F06AFA124B15
:1030A00012486361C9E7C0469461FF1FD441FF1F06
:1030B00081370000595953005959832070BA0011C3
:1030C000E1410011A061FF1F59590000A261FF1FDB
:1030D000830500009541001150BA001182150000CF
:1030E000B861FF1F871300009D42001160BA0011F4
:1030F000002370B51A4E1B4C30006361637401F0FD
:103100007DF9402323744B2B0CD9CC233821AC22DE
:1031100030009B01217401F02CFA00280AD0002510
:1031200025740CE0FFF76CFF051E08D1237C0433E7
:10313000DBB2E7E70C4B0D4D63610D4BE381236878
:10314000002B08D1002D06D00C222900200008F009
:10315000F3FB2B7B6374300001F08EF970BDC04629
:10316000D441FF1F9461FF1F3542001140BA001186
:10317000AAAAFFFFF7B5164B0192C318021D002043
:10318000009388235B05D3181B685C1C1AD09CB283
:10319000402C18D88D781E0CAC466746CD782D0291
:1031A0003D43AE4206D1019800280ED110000C70AC
:1031B000240A4C7003249BB20733A343D218009B0C
:1031C0009A42DED3FEBD4432F9E71000FAE7C0466A
:1031D000FC0F0000802213B503000324019189B283
:1031E000520107319B18A14304305A1A88235B050A
:1031F000C3181B68591C03D190429241104016BD60
:1032000099B2402907D80B000733A343C018904256
:10321000ECD30020F3E74430F9E7134B134A1B6863
:10322000126810B5FA24934201D81A00F824104B02
:10323000E4021B689A4210D813000E4A12689A42A0
:103240000ED3013307D1F823DB029C4203D10A4994
:10325000054808F071F9200010BDFC24E402ECE7F9
:10326000FE24E402F7E7C04600C0071100D00711B2
:1032700000E0071100F00711FFFFFF7FF0B59BB0E2
:10328000150004900391402A00D9A0E006AB5980B4
:103290001A80FFF7C2FF0400042816D9002206A9ED
:1032A000FFF768FF052810D906AB1B88AB420CD18D
:1032B000002D07D0514B2A000499C01808F05CFA81
:1032C000002802D101201BB0F0BD06AB1D802000FC
:1032D0000699FFF77FFF041E7BD1069B0793FFF73C
:1032E0009CFF80235B01C618802307001B039E42BE
:1032F00001D3F826F60288235B05F31801931B68B7
:10330000013302D0019808F067FA3D49019808F0AE
:1033100013F93B1D0293331D05938822029B52052E
:103320009B181B6808935A1C3CD044219AB2009108
:10333000402A04D80320D11D814389B2009103990A
:103340001B0C8B4224D0402A22D80122300008A92D
:10335000FFF710FF021E1BD1380008A9FFF70AFF74
:103360000400042831D9009A059B9B188022520141
:10337000B218934240D288235B05C118009A09A86D
:1033800008F0DAFA1D4B009A09A9F01808F01CFAA7
:10339000009A029B9446634402931A4B029AFB18CC
:1033A0009A42BAD388235B05FC1821680198013939
:1033B00008F0C2F8200008F00FFA039A07AB5A8011
:1033C00030000799FFF706FF0400002C03D100200E
:1033D00079E70428FBD988235B05E018069908F0F3
:1033E000ABF80323EA1C9A4300D16BE7034B049923
:1033F000E01808F0E9F965E70424ECE7040000119F
:10340000FFFFFF7FF80F0000F7B505001400402A0A
:1034100021D8002701AE71803780FFF7FEFE042817
:1034200016D93A003100FFF7A5FE042810D93688D6
:10343000BC420BD0BD4209D0221CB44200D9321C80
:10344000064B92B2C118280008F076FA30B2FEBDE1
:10345000C04300B2FBE703204042F8E7040000113C
:1034600037B5042204000D0001A81649FFF7CCFF70
:10347000020004280BD1019BA34208D3AB4204D025
:10348000104901A80195FFF7F9FE01203EBD0E4C41
:1034900023682000019308F09FF901992000013969
:1034A000019108F049F880235B01E418074B9C4226
:1034B000EED10422034901A80195FFF7DFFE0020A9
:1034C000E4E7C0465555000000C007110000081190
:1034D00030B589B008F060F910226946254807F038
:1034E00043FF254B009A9A420ED1019B029A0F2B63
:1034F00033D8002101240698013B08D2002900D0CE
:103500000292029B013331D10023029325E0551C26
:10351000F2D102002100EFE710341022200004A9AC
:1035200007F022FF029B013301D1069B02938823FF
:1035300004995B05C918059B06981A03120B0491A0
:103540000592814203D02B4201D108F0F5F9019B8D
:10355000013B0193019B002BDED1029B002B03D08A
:10356000049304984168084709B030BDE025014C38
:103570002D03EFE700000111504859368022F8B5BD
:10358000964C974BD200002120001C6007F004FFEE
:103590002300944A88331A60934B1A786A23002ACE
:1035A00000D01133E3620A232365904B37221B7846
:1035B0000820A3638E4B2118E361102323628D4BF7
:1035C0003B256361C823DB00A36123008C331A60B1
:1035D0002823013AE26320646364CA67043A211D28
:1035E000CA672100BC310D602100C0310860210094
:1035F000C4310B6021000635CC310D602100083D3F
:10360000C8310D602100D0310A602200D432106030
:103610002200D832136022000227E0322100176016
:103620004222DC310A6021001B3DE4310D602100A3
:10363000E83108602100EC310B6023000521F433F0
:1036400019602300F0331A602300183290331A6097
:1036500023009433186023001E3A98331A60AF2376
:10366000DB002360644BFA262363644B644DE36004
:10367000644BF031A3642300FF31FC33B600A1603A
:1036800021611E60A5627325E5656D3D6565A565D3
:1036900096255D4AAD00E264666258606766A5667D
:1036A00000270925A767E566584F594D6067200038
:1036B0002567E2673A6015279C30676007001A208B
:1036C00038602000A0300700212038602000A8309A
:1036D00007004C4838602000F83006602600642758
:1036E000A436376026005F3FAC3637602600033FC4
:1036F000B03637602600C637B4363760260000275C
:10370000B836376038269E60424E96205E64424E40
:103710005A66DE61414E9A645E62F53EFF3E9E62ED
:103720001E269A67354A8000DE661F675F67DD6583
:103730001D661862DA67BE23394A5B00E250394BD6
:10374000D838235004302250C4225200A350C6233C
:10375000E4205B00E1500433334AE1503349344BF9
:10376000D1603449800019503349E938FF38195085
:1037700032490430195032493248D161324911631B
:10378000324951631900F4310860CE2030494000BD
:1037900011603049195019002F48F83108602F493D
:1037A000D16582212E4A89005A501A002D490832CB
:1037B000D1671A002C49B432116088212B4A890044
:1037C0005A501A002A49883211602A4ADA6407F0EE
:1037D00053FF012007F0A8FFF8BDC0460004FF1FFB
:1037E0003064FF1F006FFF1F0444FF1F4A0AFF1FC2
:1037F0003A07000080C3C9019A020000DC050000FE
:103800006A18000050C3000088130000F009FF1F71
:10381000204E00006509FF1F68100000C409000069
:1038200040420F0010270000FC00FF1F751CFF1F07
:103830000000FF1FC92CFF1F5130FF1FE92EFF1F83
:103840003520FF1F2527FF1F5120FF1FFD21FF1FD0
:10385000C11FFF1F4929FF1F312AFF1F8D19FF1F9D
:103860005528FF1F7925FF1F8525FF1FC11EFF1F3C
:10387000791FFF1F391EFF1F0223F0B50124624D7F
:10388000624E2B70624B91B01C70624F0393336891
:1038900000210420BB7006F043FC042006F03AFB34
:1038A0000023984205D0BA78552A02D0332A00D096
:1038B0009DE03360042006F0ADFD07F07DFEFFF7CC
:1038C0005DFE07F0C1FD1F2201240021524B10AE06
:1038D0001A70524B1C70524B1970524B196891431D
:1038E000163A0A431A60602219689143403A0A4323
:1038F0001A6007F089FD07F0D7FD4B4B9847C120B0
:10390000FF214A4B80001A588A431A50C522920060
:1039100098588843BF390143995098584449084002
:103920008021C9010143802099509958C00509029E
:10393000090A0143995080213E48490107F094FE4D
:10394000032322003C49019400933C4807F084FE85
:103950002C223B4905A807F0EFFF05AC61782078E1
:10396000023406F0F7FAA642F8D1364C11200021B5
:1039700006F004FC2268344B03201A40A023DB022B
:1039800013432360802322689B041343236022682F
:103990002E4B1A4080239B03134323602C4A2D4B4C
:1039A000934200D8012007F017FD07F005FF8023A0
:1039B0002268DB0413432360287807F0BDFE039BD5
:1039C0001878C0B207F068FD07F06EFE22490420A7
:1039D00007F0BAFE06F0EAFC00F040F800F000FE46
:1039E00000F0A8FE00F004FA002011B0F0BD009332
:1039F0002100194A042007F047FE8023DB059C6262
:103A0000FFF766FD56E7C0464A0AFF1F34F0004044
:103A10000444FF1FC461FF1F480AFF1F490AFF1F1C
:103A2000680AFF1FBCF00040E1A2000000E100E0D6
:103A3000FF00FFFF0844FF1F8C56FF1F0854FF1FA5
:103A400068B9001114F00040FF7FF8FFFFFF9FFFEF
:103A50000080FF1F006FFF1F3B000108002210B510
:103A60001100112007F010FD10BD0000002370B5FB
:103A70000925334E334C3362E3681120AB43E360D6
:103A800007F002FF112007F07FFD112007F03CFF37
:103A90004023226811201343236080236268DB02E5
:103AA000134363608023A2681343A360A368264A7C
:103AB0001340A3608023A2689B0113431022A360DC
:103AC000236C934323640123226C1A4322648022D3
:103AD00052003262216B1D4A11402163616B11401B
:103AE0006163A16B1140A163E16B0A40E263E2688C
:103AF00017490A40E260174A11680B43136007F048
:103B00006BFDFD21144B154A89005A508023C720B4
:103B1000626B5B0313436363E36880001D43104BD8
:103B2000E56019580F4A1140802212020A431A50C8
:103B3000802292051A6008220B4B5A6370BDC04662
:103B400000F000403CF00040FFFFDFFFEFFFEFFF21
:103B5000FFFF7FFF003800400000FF1F5118FF1FCC
:103B600000E100E0FF00FFFF0000054070B5284CB9
:103B7000238C002B23D0228A002A21D1DA00238231
:103B80006382A382E38223836383A383E38322602C
:103B90006260A260E2601F4D1F4A6420EB80934286
:103BA0000AD8FA220020D200934205D91B4A0A21E2
:103BB000981807F021FCC0B200232872238470BD3E
:103BC0000720E11CCA7F01320240CA7705D10325D4
:103BD000201DC17F01312940C17708325200A35214
:103BE000002321001A00088A01321B180231082A1A
:103BF000F9D1221DD27F9200A350626823689B18DE
:103C0000A2689B18E2689B185B099BB2C3E7C04699
:103C10000461FF1FAC61FF1FB70B000030F8FFFF0E
:103C200030B503A804880B20002C0ED14968074D3D
:103C300008784978090201430A20A94205D10121E7
:103C400020001980024B1B7A137030BD192A000026
:103C5000AC61FF1FF7B5150008AA16884A680F4F18
:103C600014785278120222430A24BA4214D1012253
:103C7000DBB2019200962A0007F0E8FA041E0BD18D
:103C8000074B1B68002B07D068782A780002104386
:103C900042425041013098472000FEBD02290000F9
:103CA0003061FF1F30B5012503790400BFB02B42FE
:103CB00011D00A49408806F035FE28420BD0084B47
:103CC00001A95B8D4D800B80064B00221B7A60881A
:103CD0000B7103F007FF3FB030BDC0462861FF1FE6
:103CE0004840FF1FAC61FF1F10B50549054806F0AD
:103CF000CFFD0421044A054806F08CFD10BDC046E6
:103D00002861FF1FFFFF000094B900114840FF1F0A
:103D100010B5024804F068FD10BDC046A53C001176
:103D2000012303700B4B1A7A4270022282709A7838
:103D3000C270DA780271032242711A7982715A795B
:103D4000C2710C2202729A794272DB7983720B2063
:103D50007047C046AC61FF1F022310B50370013BE2
:103D600043700533837010330371443B43712A332E
:103D700083714433C37100230372064B04001B8814
:103D800043720A30FFF7CCFF831D0A30C0B2E370E4
:103D900010BDC046AC61FF1F10B5142007F08CFBAE
:103DA000124B14220021186007F0F6FA002007F0E9
:103DB0009BFD012007F040FB022007F025FD0320BA
:103DC00003F0B6FF042005F0CBFF052003F0F4F963
:103DD000062003F0C1FE072001F058FA082006F083
:103DE000F9FC092001F034F810BDC0463461FF1F12
:103DF00007F0AAFB012007F08FFB07F0ADFC0000E5
:103E0000094B10B50400984205D0012904D12000C7
:103E1000064906F03DFD10BD0229FCD1013904F030
:103E2000A1FC0028F3D0F6E7FEFF00005A61FF1F57
:103E300070B50D7A100004AA2C00168810221440C8
:103E4000154220D1002E20D10A78022A18D14A68C2
:103E5000517815780E4A09022943914205D00D4A3E
:103E6000914209D01C800A2404E014220A491A80D5
:103E700007F062FD200070BD0C2208491A80F7E7A8
:103E80001C800124F6E70824F4E70B24F2E7C0467F
:103E9000F3FF0000F4FF00009042FF1F8CBA0011F6
:103EA00010B504000749084806F0F2FC074804F082
:103EB000DBFB0020E40704D50721054A054806F08E
:103EC000A9FC10BD5A61FF1FFFFF0000013E001159
:103ED000D8B900118C40FF1F00B50C4BBFB01A7849
:103EE0000B4902A800F0E0FC6B4680B2D8800028A5
:103EF00009D06A46074B01A91B889380064B002214
:103F0000188803F0EFFD3FB000BDC0463861FF1FC9
:103F10003961FF1FE640FF1FF041FF1F00B50C4B4A
:103F2000BFB01A780B4902A801F022FD6B4680B29F
:103F3000D880002809D06A46074B01A95B8D938081
:103F4000064B0022188803F0CDFD3FB000BDC046EF
:103F50006261FF1F6361FF1F8C40FF1FF041FF1F65
:103F6000F7B50E00377A1C0008AB11003D001A8827
:103F700020231D401F423CD13378022B3BD1736874
:103F80001F785B781B023B431E4FBB4208D01E4F7D
:103F9000BB4214D01D4DAB4221D00A252800FEBDE6
:103FA000002A2AD1142C2AD82200F06807F0C4FC79
:103FB000174B1C70012CF1D9FFF7B0FFEEE7002A78
:103FC0001BD1202C1BD82200F06807F0B5FC114B48
:103FD00004211C70104B187807F0A6F9DEE7E3B255
:103FE0000124009201940A00310007F02FF9050026
:103FF000D4E70825D2E70125D0E70B25CEE70D252C
:10400000CCE7C046F3FF0000F4FF000002290000E7
:104010006261FF1F3861FF1FE461FF1F332310B58A
:10402000040003700A220749013007F085FC064BA3
:104030000F201B681A0AE37222731A0C1B0E62739C
:10404000A37310BDAC61FF1FD461FF1F30B5012504
:1040500003790400BFB02B4213D00B49408806F00F
:1040600061FC28420DD06A46084B02A81B88938049
:10407000FFF7D4FF6B46D8800022608801A903F0C7
:1040800031FD3FB030BDC0465A61FF1FE640FF1F03
:1040900010B5024804F0A8FB10BDC0464D40001109
:1040A00070B5160004AA148805AA15784A685078D5
:1040B000117800022A4A0843801805284BD807F0D7
:1040C0009BFB03131E29343F0720032C0BD804222B
:1040D000121BAA4200D92A0022491A80300009196D
:1040E00007F02AFC002070BD0720112CFBD81222FB
:1040F000121BAA4200D92A001B491A80EEE70720AA
:104100000E2CF0D80F22121BAA4200D92A00174900
:104110001A80E3E70720032CE5D80422121BAA42E9
:1041200000D92A0012491A80D8E70720032CDAD8D0
:104130000422121BAA4200D92A000E491A80CDE798
:104140000720032CCFD80422121BAA4200D92A0030
:1041500009491A80C2E700220A201A80C3E7C04634
:10416000DCD5FFFF23BA00118061FF1F13BA0011D5
:104170000EBA001109BA001104BA001110B50D21D0
:10418000024A034806F046FB10BDC046F8B90011CC
:10419000FC40FF1F13B5104C0423217C01AA00F042
:1041A000ADF9002815D16B469A88236852BA92B2AD
:1041B0005343228909491B0C9B184B806B46DA88B4
:1041C000636852BA92B2534362891B0C9B188B806E
:1041D00016BD0120FCE7C0469461FF1FAC61FF1FC4
:1041E00013B5124C06236A46217C00F087F900289B
:1041F00019D16B461988236849BA89B24B43218982
:104200000B4A1B0C5B1853806B46D97803335B78E1
:104210001B020B435BBA61689BB24B4361891B0C69
:104220005B18938016BD0120FCE7C0469461FF1F18
:10423000AC61FF1F37B5174C07236A46217C00F09D
:104240005DF9002824D16B461B787F2B20D86B4664
:10425000DD78F0232A041B031A406B469B880E4925
:104260005BBA9BB21A4323682D09534322891B0C66
:104270009B184B806B465A789B7812031B011A439C
:1042800063682A43534362891B0C9B188B803EBD95
:104290000120FCE79461FF1FAC61FF1F7FB5022680
:1042A000154C0022217C03AB0096050000F0F8F8C5
:1042B000002802D0012004B070BD0E23217C012211
:1042C000280000966B4400F0EBF80028F2D16B4612
:1042D0009A892368D2BA5343228908491B149B1830
:1042E0004B806B46DA89636852BA92B25343628953
:1042F0001B0C9B188B80DEE79461FF1FAC61FF1FD6
:1043000070B5184C237C002B0FD0382B0ED1164DD6
:10431000280000F073F8CC23AC222800217C9B01FC
:1043200000F027F9280000F0A7F870BDE3890F4AD4
:10433000934209D10C4D280000F060F800222800BB
:10434000217C00F005F9EDE7094A9342EDD1064DD5
:10435000280000F053F890222800217C920100F000
:1043600026F9DFE79461FF1FD441FF1F830500009A
:104370008320000070B5144C237C002B1FD0636990
:10438000002B1CD0114D280000F038F8636928007C
:1043900098470400280000F06FF8002C10D10C4B57
:1043A0000422995E002905DA9C801A8801321A805D
:1043B000200070BD074A9142F7DD9A80F5E701249D
:1043C000FEF796FEF4E7C0469461FF1FD441FF1F3D
:1043D000AC61FF1F0F27000010B58024064AA4001F
:1043E0001168436B234205D113685B1A032BF8D97C
:1043F000012010BD0020FCE76008FF1F70B5C179E7
:1044000005000C00631E9C411A4BE402E4184900AD
:104410000460C9B2007905F0E7FEE97968794900DE
:104420000131C9B205F0E0FEE8790930C0B207F009
:104430006BFA0023E36661332360AA795B3B002AB1
:104440000ED022689A43023B134323600A23E361A0
:104450000733236200232363A3630133E36370BD47
:1044600022689A4302231343236046236361063381
:10447000A361EFE70050004070B500250400036819
:10448000DD66C0790930C0B207F0FEF92900207955
:1044900005F046FE2900607905F042FE70BD00007F
:1044A000F8B51E0006AB1D78002304681700E3660C
:1044B000616007F071F901238022E3662B00276118
:1044C0005200013B08D207F007F908200A4A116898
:1044D000002D03D12800F8BD2261F2E7236F0342CB
:1044E00003D02369013D3370013613685B1A032B37
:1044F000EED90125EEE7C0466008FF1F70B51C002D
:10450000002305681600EB66696007F045F9012392
:104510008022EB6623005200013B08D207F0DCF852
:1045200008200A4A1168002C03D1200070BD2A61BE
:10453000F2E72B6F034203D02B69013C3370013645
:1045400013685B1A032BEED90124EEE76008FF1F06
:10455000002370B504681500E366616007F01CF97C
:104560000123E366256107F0B7F82000FFF734FF69
:1045700070BD70B51D00002304681600E36661601D
:1045800007F00AF90123E36626610F33626B1A42D2
:10459000FCD02B0A23611023626B1A42FCD0EDB2CF
:1045A000256107F099F82000FFF716FF70BD002382
:1045B00070B504681500E366616007F0EDF801234B
:1045C000E3662B0A23611023626B1A42FCD0EDB222
:1045D000256107F081F82000FFF7FEFE70BD0000A6
:1045E00010B5084CE368002B08D18022064B52021C
:1045F0001B689B186360054B1B68236007F034F948
:10460000A06010BDD461FF1FC8F00040CCF0004096
:1046100070B5184A936A916A9942FBD116498A6823
:104620009A421FD39A1A8B60144B0126186893B2D2
:10463000D202D20E4343424300204C681B0A1B198E
:1046400012029B180E4C0A684B60551CA3420CD8F2
:10465000002801D04B600A600A4A136008680A4BC0
:10466000186070BD581E821ADDE7084A30009B189A
:104670002A00EAE700F00040D461FF1F140AFF1F80
:1046800040420F00C8F00040CCF00040C0BDF0FF39
:1046900070B51F4C23793F2B01D93F2323711D4B4C
:1046A00022791A701878C0B206F0A6FF18231A49AA
:1046B0001A4A0B801A4913800B805380A379194939
:1046C00080200B800C21938001334B43164D191C25
:1046D0000001834200D9011C2980D1806379002B1D
:1046E00011D101336371237A012B01D80223237284
:1046F0006279237A0D4853430A21584306F07CFE21
:104700000B4D286070BDA02BEDD9A023EAE7C04671
:10471000C861FF1F480AFF1FEE41FF1FB043FF1F84
:10472000EC41FF1FEA41FF1FE841FF1F710200003B
:10473000B861FF1FF8B519210020FEF791FE114C5A
:10474000011E114D09D10C22104BC1CBC1C4280050
:1047500006F022FEFFF79CFFF8BD0C2220000C495A
:10476000FEF752FE0C2802D0084B43CB43C40C2268
:1047700028000849FEF748FE0C28EBD00C22002147
:10478000E5E7C046C861FF1F9461FF1F80BA0011B2
:10479000FC0C0000F50C0000F0B51D4C8022A54477
:1047A0000400882069465201400507F095F89022E0
:1047B00012016A441300200032C832C316C816C35F
:1047C0008023144C144FA6689B033343A3603B60C3
:1047D00006F0A2FD8823A0685B05C01806F0FCFF68
:1047E0000025882329008022A0685B05C018401995
:1047F0006944520006F0E8FF80230135FF355B0174
:104800009D42EED1A6603E60044B9D44F0BDC04683
:10481000FCEFFFFF2043FF1F9808FF1F041000005C
:10482000F0B5040087B0002825D0684606F08CFD5E
:104830001B4C022806D106226946200006F09CFF88
:10484000002816D06946002301250F262F00E25CC0
:10485000013310091030874038002F003240974054
:104860003A0002434A610439062BEFD16846FFF74C
:1048700093FF07B0F0BD182269460A4807F02CF8EC
:104880006A46A300D358013305D01822FF21684699
:1048900006F082FDEAE70134062CF1D1E9E7C046D3
:1048A0006509FF1F00090011F0B5002504000E0086
:1048B00085B0AA4200D183E04B1C087801934B7865
:1048C0008978377909021943F3783F061B040B43B3
:1048D0001F43039720706570252800D193E033D8DB
:1048E000112813D806F0A8FF66000D010D010D0177
:1048F0000D01A700B500AE000D010D010D010D0168
:104900000D010D010D010D01E7000701232800D164
:10491000C0E0DB2800D016E1042A00D8A9E0102569
:10492000052A05D0551F2A003800711D07F004F82C
:1049300005223100200006F0FFFF2A003900601D2B
:1049400006F0FAFF05353BE0562856D010D833283C
:1049500000D19AE0552836D02628DAD1894B290093
:10496000132218001D0006F017FDFEF7C1FB59E0E9
:10497000712800D174E0722800D17DE0DC28C8D114
:10498000022A00D875E07378BFB26370B378A37061
:10499000032A05D0033A390092B2F01CFEF76EFCF0
:1049A00010223900E01CFEF72FFDC51C002807DA95
:1049B00060705CE00C222000734906F0BDFF0C25FE
:1049C000280005B0F0BD013A704D0C2A13D8002A1A
:1049D0000AD02800019906F0AFFFFFF759FE0C221C
:1049E00028006B49FEF74AFC29000C22601C06F0E7
:1049F000A3FF0D25E4E70C22EBE7644D654B2A008D
:104A000043CB43C2E9E7013A5E4D0C2A11D8002A94
:104A100008D00199280006F08FFF0C2228005E497B
:104A2000FEF72CFC29001322601C06F085FF1425DC
:104A3000C6E70C22EDE706225849601C06F07CFF11
:104A40000625BDE712225649601C06F075FF1325A6
:104A5000B6E708225349601C06F06EFF0925AFE750
:104A60007178F02905D8504B188801F0DDFB02253C
:104A7000A6E7FF236370FAE74C4B012A03D0727854
:104A80005A706270F3E75B78F4E72000FFF7C6FA2C
:104A9000050095E7042A04D9454D2F6006F0E4FE91
:104AA000A860FFF7B5FD0422039003A9601C06F07F
:104AB00043FF052584E73F4D062A15D90622280025
:104AC000019906F059FE00280ED00622019928000F
:104AD00006F032FF062238492800FEF7CFFB0123FB
:104AE000324A51780B43537029000622601C06F0AD
:104AF00023FF072564E7012ABBD07078FFF790FEFB
:104B0000B5E7012800D004E7931E2C4F132B06D8DD
:104B10007378002B0BD100F009F900F03FF9284B16
:104B200039001D78601C6A1E06F006FF48E7551E16
:104B30002A000199380006F0FFFE38002149AAB288
:104B4000FEF79CFBE9E7DA2893D1042A91D9082AD9
:104B500015D9B37972791B021343F27912041A43FF
:104B6000337A1B0613433B603B680522310020006B
:104B7000039306F0E1FE0422601D03A96CE7FE2307
:104B80006370F1E79461FF1F8CBA0011C861FF1FC9
:104B9000FC0C000080BA0011F50C0000A061FF1FA2
:104BA0008061FF1F2443FF1FF041FF1FC461FF1FEF
:104BB000D461FF1F6509FF1FADAC0000C563FF1F77
:104BC000C363FF1FAEDE000070470000020010B597
:104BD000094B0A32094C92B2DA815A8298811882C2
:104BE000207802F087F90422054B012120781A7001
:104BF00006F09AFB10BDC046AE42FF1F0E64FF1FB9
:104C00000D64FF1F013870B5042809D806F0F4FDC3
:104C10000309230812001E4B0221187806F084FBBA
:104C200070BD1B4B0821187806F0EEFC0022194BD2
:104C30001A72F5E780220024164B154D52001A8196
:104C4000082128781A68DC7206F0B6FB2100287863
:104C500006F0AAFCE4E70E4B0821187806F0D4FC15
:104C60000D48FFF779F80D4B0D4A9B7993800D4A5B
:104C700013800022074BDA720132FF321A810A4B8D
:104C80005B78002BCCD0094A136006F065FBC7E7C0
:104C9000E461FF1FB861FF1FF941FF1FC861FF1FDB
:104CA000B043FF1FEA41FF1FC461FF1F34F0004003
:104CB00010B5002904D1042802D10D3005F05EFAA8
:104CC00010BD000010B501290ED104280CD10D3003
:104CD00005F054FA054B1B78002B05D02622044B17
:104CE00004485A72FFF772FF10BDC046E663FF1F0B
:104CF000B861FF1FC40900000300F0B50A4D8E180B
:104D0000B14202D152008018F0BD0C782F682409FE
:104D10003C5D0F271C700C7801313C402F683C5DD6
:104D20005C700233ECE7C046E441FF1F0D22124BDA
:104D300010B51A700C23114C11492370093A033B2A
:104D40001048637006F0F8FD2D2301220E490F482C
:104D5000A371FFF7D1FF01220D49FFF7CDFF01221B
:104D60000C49FFF7C9FF030000200B49020018702F
:104D7000FEF784FA10BDC046E263FF1FC363FF1F46
:104D800023BA0011C563FF1F6709FF1FCA63FF1F16
:104D90006609FF1F6509FF1FAEDE000070B5134CEA
:104DA000142220001249FEF72FFB431E114D132B36
:104DB00019D8AB78002B16D0431C2B7009236B70CD
:104DC00000230019037028780B4B01302900C0B272
:104DD000187006F099FC297822000139C9B2002028
:104DE00005F036FC70BDFFF7A1FFECE7C563FF1FC0
:104DF000AEDE0000C363FF1FE263FF1F10B5114B5F
:104E00001A781870002A0ED000280BD10E4B1A7891
:104E1000062A07D85423D340DB0703D50B4B187859
:104E200002F068F810BD0028FCD0074B1B78012B5E
:104E300002D0033B022BF5D8044B0121187806F071
:104E400073FAEFE7E663FF1F0D64FF1F0E64FF1F99
:104E500070B54D4E4D4A4E493070042005F084FA2D
:104E60000021112005F08AF9112005F06BFAFEF7F8
:104E70003FF906F079FB032246494748FFF73CFF1C
:104E80002D24030004221C7044490130FFF734FF35
:104E900030230470424D434C437083702E3B0622F6
:104EA00020004149EB87FEF7AFFA062813D0200017
:104EB00006F04AFA022809D00321200006F0CCFCB3
:104EC0008D23E3706E3B237119336371062220003A
:104ED0003549FEF7D3F9354B1B68FC335C64FFF7AB
:104EE0005DFF0020FFF78AFF314C324A0121324B2F
:104EF0001278207801F0C0FF304A314B127800213F
:104F0000207801F0B9FF01222E4B1A702E4B9B78AE
:104F1000552B31D12D4B3B325A722D4B2D4AAB8143
:104F2000EA812B826A822021307806F08DFC0120F4
:104F3000404205F0D9FB0120404205F075FCFFF727
:104F40001DF9FEF7D1FE00F0ABFC01204042FEF758
:104F5000A7FF012006F060FCF02001F049F90121D3
:104F6000307806F0E1F9307802F020F91A4806F0BE
:104F7000A3FCFEF77BFD70BD6422184B5B795343A5
:104F80001A000A32CBE7C046E461FF1FB14C0011A2
:104F9000C54C00112443FF1F8061FF1FA061FF1F4C
:104FA000AE42FF1F6509FF1FADAC00003064FF1F5C
:104FB0000E64FF1F1842FF1FF941FF1FE263FF1F2E
:104FC000C363FF1FB463FF1FC461FF1FB861FF1FEE
:104FD000C4090000CE090000E661FF1FC861FF1F81
:104FE000F8B50A0020230D001A4019425DD05A4B33
:104FF0001B78002B42D0FFF70BFB584B584C594EF7
:1050000099686268737A8A1ADB039A4202D36160F4
:10501000FEF72CFD327A217A531EDBB2994230D151
:10502000FFF76EF9637A002B25D0013BDBB2637288
:10503000002B20D14C4B9B78552B01D106F08CF9DD
:10504000E37A002B12D00023A27AE3729A4202D0B4
:10505000A372FEF78BFD454A454F13883800013394
:105060001380FEF779FE390006F086FA6423707922
:105070005843FFF7ABFD237A0133237220206840A9
:10508000F8BD9142CED300272772FFF773F9A37AB8
:10509000BB4202D0A772FEF769FD354F3800FEF71C
:1050A0005BFE390006F068FABCE70BB2002B0ADAA7
:1050B000304B187806F048FC002801D006F014FBAD
:1050C00080200002DBE70224214206D0244B01208D
:1050D0001A72FFF793FE2000D1E70B071BD5FFF7ED
:1050E00097FA1E4B1E491F4C98684A68637A821AC9
:1050F000DB039A4202D34860FEF7B8FCFFF73AF9A7
:10510000FFF7FEF800F0E6FB2368DB0701D5FEF7AA
:10511000BFFF0820B3E7CB0609D5FEF727FD0E4BEE
:105120001B78002B01D1FEF7F3FD1020A7E7012427
:10513000214209D0104800F06DF806F075FA210000
:10514000112005F01BF8C6E7042408002040214286
:1051500096D0FEF7C1FEBEE7E663FF1FD461FF1FD6
:10516000B861FF1FC861FF1FC461FF1FAC61FF1F53
:10517000F941FF1FE461FF1FDC41FF1FF0B51B4B2E
:105180001B4F1B883A8804001A4E1B4D85B09A426B
:105190000DD832889A420AD3184B1A882B889A4223
:1051A00005D1174A174B12881B889A421BD005203D
:1051B00001F074F83B8802AA138033880190538071
:1051C0002B88114D93800F4B02A91B88D3800F4B66
:1051D0002A78188802F090FD0D4B08212878019A52
:1051E0001C7006F0A1F905B0F0BDC046B263FF1F08
:1051F000EE41FF1FEC41FF1FEA41FF1FB063FF1F9D
:10520000AE63FF1FE841FF1F0E64FF1FF041FF1F49
:10521000AC63FF1F13B50C4B1C78002C11D1002878
:1052200001D00A4B18600A4A0A4B11780A4A1078D2
:105230000A4A01920A4A0092002205F001F9200070
:1052400016BD1124FBE7C0460D64FF1FA863FF1FB6
:105250000C64FF1FFC63FF1F0E64FF1FE863FF1F4A
:10526000EC63FF1F10B5064B12201B78052B06D1EF
:10527000044B13221988044B187801F0EBF910BD88
:105280000D64FF1FF041FF1F0E64FF1F10B50024C7
:105290000122114B52421870104B1C70104B1A8097
:1052A00001F084FF04220F4B21001A700E480C32CB
:1052B00006F05AFA102221000C4806F055FA07228F
:1052C0000B4B1C600B4B1C700B4B1C700B4B1A7068
:1052D0000B4B1C7010BDC0460E64FF1F0D64FF1FFA
:1052E000F041FF1F0C64FF1FFC63FF1FEC63FF1FF7
:1052F000E863FF1FC263FF1FC163FF1FF241FF1F6F
:10530000C063FF1FF8B5174C0600257806A81424C3
:105310000078052D23D1B41F134FA5B21824BD4228
:105320001DD88D1FADB2BD4219D8FA256D00AA4215
:1053300015D21D000D4F0A3DADB2BD420FD80C4C29
:1053400026800C4C21800C4900240A800B4A1380D3
:10535000FFF714FF0A4B0421187806F055F92000D6
:10536000F8BDC0460D64FF1F790C0000750C0000ED
:10537000EE41FF1FEC41FF1FEA41FF1FE841FF1F05
:105380000E64FF1FF0B50BB20D0089B0002B00DBDF
:1053900070E1A44E307806F0D7FA041E50D003789E
:1053A000A22B00D122E1D02B1AD0912B45D14378EA
:1053B0000E2B42D19C4B82889A423ED19B4A8368F5
:1053C0001278052A39D1032018567F2835D0984BFA
:1053D0001B68002B31D05B68002B2ED098472CE047
:1053E0008078072829D806F007FA0428183F3F7468
:1053F000A8D86378002B0CD101218C4B19708D4BF0
:105400001A78002A5BD08C4B307801F035FD0028EB
:1054100055D00722854B1A7051E061780029F8D1E8
:10542000E378002B11D0854A854B1278307801F053
:1054300023FD60706378002BEBD1200006F054F957
:1054400080200002684009B0F0BD784B1B78022B29
:10545000F3D00121307806F03FF80028EAD101218D
:10546000307805F061FFE5E76378002BD1D16F4F0D
:10547000032807D13B78052B02D101333B701EE096
:105480000223FBE76F4B1A886F4B0293002A0BD065
:105490001B78002B03D00121307806F045F83B78CB
:1054A000062B04D1013BE9E7029B1A70F7E7042BB6
:1054B00041D10121029B3078197005F035FF5C4B1A
:1054C0001B68002BB9D01B68002BB6D0574A107848
:1054D00084E76378554F002B27D10622211D5B48B6
:1054E00006F02AFA62895A4B5A491A80A2895A4B05
:1054F0001A80E3890B800521397058490A80584A7F
:105500001380228A574B1A80574B1B78012B09D1E5
:105510001F2000F0C3FEFA2292004243042130789B
:1055200006F002F80022484B75E7312B00D070E7F7
:105530000022454B1A700323A0E7062200214348AE
:1055400006F012F90023454A04211380444A3078BA
:105550001380444A138006F057F80821307806F08B
:1055600053F8A379083B5A425341304A033313702E
:10557000304B1B78002B06D0334B30781A78002A3A
:1055800006D001F0B7FC0122314B52421A8096E757
:105590000121197005F0C8FEF5E70821307806F002
:1055A00033F86378002B00D047E72C4B2D4F029344
:1055B000E388029A04211380294B307803932389CE
:1055C000039A138063893B8005F086FF002800D092
:1055D00033E7264B1B68002B00D12EE70399029876
:1055E0003A88098800881B68984726E74379132B77
:1055F00000D022E70389012B0AD11D4B1B78022B17
:1056000006D10821307805F0FFFFFFF72BFE14E7E5
:10561000052000F043FE08210200307805F084FFE9
:105620000BE7C0460E64FF1F051400000D64FF1F4A
:10563000A863FF1F1842FF1FF941FF1FE263FF1F0E
:10564000C363FF1FE463FF1FE663FF1FB563FF1F14
:10565000F041FF1FBC63FF1FBE63FF1FB263FF1F4C
:10566000B063FF1FAE63FF1FB463FF1FA463FF1F80
:10567000AC63FF1F8020C001014200D0E2E6CB07EF
:1056800031D5324B1B78002B1DD0314E05AC337811
:10569000052B1AD1023B23702E4B21001B7823725D
:1056A0002D4B1B7863722D4B187801F089FB002875
:1056B00009D007202A4B30701B68002B03D01B68D1
:1056C000002B00D098470120BCE60E20254B062277
:1056D0001B7825492370254B1B78637002ABC018DB
:1056E00006F02AF9D8E7022308001840194209D029
:1056F000174B1B78052B03D11D4B188805F0CCFFE9
:1057000002209FE60424214203D0FFF737FD20004A
:1057100098E6082308001840194200D193E6154B7B
:105720001C78012C03D0022C0DD008208AE6124BE5
:10573000124A134913481B8812880988008800946C
:10574000FFF7E0FDF1E7FFF78DFDEEE7E663FF1FF2
:105750000D64FF1FF241FF1FC063FF1F0E64FF1F98
:10576000A863FF1FC263FF1FF341FF1FC163FF1F39
:10577000F041FF1FAC63FF1FE841FF1FEA41FF1F1D
:10578000EC41FF1FEE41FF1F10B502A804880B205B
:10579000002C10D1496808784978090201430C4867
:1057A000814209D1022119800A4B59881170DB7896
:1057B00000205BB2537010BD074C0A20A142FAD101
:1057C00002211980034B998811705B79F0E7C0467C
:1057D0006E2A0000AC61FF1F6F2A0000F7B51500AC
:1057E00008AA16884A680F4F14785278120222438A
:1057F0000A24BA4214D10122DBB2019200962A0097
:1058000005F024FD041E0BD1074B1B68002B07D0AD
:1058100068782A780002104342425041013098478C
:105820002000FEBD022900002064FF1F30B50125C5
:1058300003790400BFB02B4225D01449408805F0FD
:1058400071F828420CD0124B01A95B8D00220B800D
:1058500002234B800F4B5B888B80608802F042F9FB
:105860000D49608805F05EF8C0070CD50B4B01A907
:105870001B8800220B8002234B80064B9B888B8069
:10588000608802F02FF93FB030BDC0461864FF1F9A
:105890001C42FF1FAC61FF1F1064FF1F7642FF1FF9
:1058A00010B5074C0749200004F0F2FF200006491C
:1058B00004F0EEFF0721054A054804F0ABFF10BDD8
:1058C000FFFF00001864FF1F1064FF1FACBA001137
:1058D0001C42FF1F10B5024802F086FF10BDC046F3
:1058E0002D5800110200F0B501270A480A4E511840
:1058F0008B1A002B00DCF0BD0824157843086840A3
:1059000038404000805B013C58406D08002CF5D1C8
:105910000132EDE7FFFF0000C6BA0011F0B5002527
:105920000F269D4200DBF0BD4C5D0709444034402A
:10593000A400A05801357840F3E70000F0B589B025
:105940006A460D000B000F27110010351C7801333B
:10595000260024093E40167054700232AB42F5D145
:105960002023024AFFF7DAFF09B0F0BDCCBA0011DC
:10597000F0B54E780B7889B036020C001700019014
:105980001E43012A61D9954B9E4200D877E001332E
:105990009E421CD1062A17D1CA788B7812021A436C
:1059A0000B791B0413434A7912061A438C4B5A6134
:1059B00000221A705A808B4A5A608B4A9A608B4A2E
:1059C000DA60002009B0F0BD88225205EEE7884B6E
:1059D0009E423CD182498B78002B00D0F6E00C2A05
:1059E00031D10F22A3789343E27812021343227934
:1059F000120413436279120613434B60E279A079D3
:105A000012020243207A00041043627A1206024313
:105A1000CA60E27AA07A1202024376484A8183423F
:105A200008D804236E49142201980B7005F084FFF6
:105A30001420C7E71201D21889235B059A42F0D8D7
:105A400001238B70BDE7022AFAD00523EAE76A4AF0
:105A500001239642E6D1FFF705FC052F0CD9E37828
:105A6000A2781B021343227912041A4363791B069E
:105A70001343624A0393136005F06EFCA1E7584D8F
:105A80002B78002B9DD1AB78002B00D1A0E02B8987
:105A900001339BB20093B34200D091E0132AD4D9D2
:105AA000CF7C8B7C3F02122120001F43FFF71AFF9F
:105AB000874200D08EE0002E3DD1E378A2781B0211
:105AC00013432279E96812041A4363791B061343CE
:105AD00003930A228B4212D1FF23A370E370237138
:105AE00063716B89002B09D1E37B227C1B021204BA
:105AF0001343A27B13431B0901336B8100226B8983
:105B0000002B8ED0002A67D1686837013818000B47
:105B10006B6900030390984205D9686105F05CFE4B
:105B2000EB780133EB7068681022A11C381805F07F
:105B30004BFE2E8145E76F89009A7B1E9BB29342F4
:105B40003AD1E278A37812021A43237905A81B04FC
:105B5000134362796C6812061A43EB680092039251
:105B6000211D0C22049305F0E7FE0120260004A964
:105B700040421036FFF7E2FE013F012F17D1009A95
:105B80000B232861824200D04CE704221C492000EC
:105B900005F01AFE042203A9686805F09DFEE96875
:105BA000039AFF23914200D13CE7F73B3AE73100EB
:105BB000FFF7C4FE1036DFE70923B742A4D831E768
:105BC000009BB34200D9FCE607232BE7022329E719
:105BD000032327E7062325E70A2323E7FFFE000028
:105BE0009042FF1F00000111FFFF0000504859368E
:105BF00001FF0000FFFF001102FF000034F0004031
:105C00009C42FF1F10B5034C0B000122210000F045
:105C10006BFA10BDC55D00110B8870B506000D0054
:105C20000224162B11D92B000322094900F05CFA3B
:105C3000041E0AD1074B2A881B88191C934200D9DD
:105C4000111C300089B200F0EFFA200070BDC04690
:105C5000F15D00113664FF1F10B54A780400013A67
:105C60000B000220012A07D80A78002A04D0052256
:105C70002000024900F038FA10BDC0461F5E001136
:105C80000A7810B50B0004000220002A04D0072275
:105C90002000024900F028FA10BDC046CB5E00117A
:105CA0000A7810B50B0004000220002A04D0092253
:105CB0002000024900F018FA10BDC046315F001103
:105CC00010B5034C0B000B22210000F00DFA10BDA3
:105CD000615F001110B5034C0B000D22210000F094
:105CE00003FA10BDD35F001110B5034C0B000F2257
:105CF000210000F0F9F910BD2D6000110A7810B5EF
:105D00000B0004000220002A04D0112220000249C6
:105D100000F0EAF910BDC0463D600011002310B547
:105D20001322190000F0E0F910BD000010B5034C7B
:105D30000B001722210000F0D7F910BD8F60001171
:105D4000002310B51922190000F0CEF910BD000093
:105D500010B5034C0B001B22210000F0C5F910BD4B
:105D6000C9600011F7B584890D0006000121002CDF
:105D700022D000238268D3561778002B1EDA0C2C11
:105D80001AD90C3CA4B2131940880093230002F0E6
:105D900086FE431E984101307B06DB0F6B703F236C
:105DA000013C1F40A4B22870AF70AC80002C07D01B
:105DB000B3680133AB6000210800FEBD0020EBE7B3
:105DC000AC60F8E70B7803704B8843704B881B0A74
:105DD00083700B79C370042070470420022B06D116
:105DE0000020537811781B02009A0B4313807047F0
:105DF0000B8803700B881B0A437002207047042035
:105E0000009983420AD1537810781B0203430B8018
:105E1000D37890781B02034300204B807047F8B57D
:105E20000D004B7801240021461C03702B788B4217
:105E300001D82000F8BD6B78B01C4F1C012B10D18D
:105E4000890069184B88022233704B88B9001B0AFD
:105E50007370691805F038FC04360434A4B2F9B242
:105E6000E4E7122359436B185A88043132705B8877
:105E700010221B0A7370691805F026FC12361234C2
:105E8000ECE770B5049D14001E00052B01D804201A
:105E900070BD637812781B0213432B80E378A278DD
:105EA0001B02134302226B802A71211D681D063ECE
:105EB00005F00AFCB2B22A81E92AE8D82800A11D1F
:105EC0000A3005F001FC0020E2E7002310B50A7853
:105ED0009A4201D8900010BD9A008A185488013364
:105EE00004705488DBB2240A4470948884709288C9
:105EF000120AC2700430EAE710B51100029C062BAA
:105F000004D004201022142B01D010BD02222271D3
:105F10004B7808781B0203432380CB7888781B02D8
:105F2000034363800431601D05F0CEFB0020ECE7E5
:105F300010B50C788B7804315C43E4B20370220016
:105F4000013005F0C1FB601C10BD0420022B06D1FE
:105F50000020537811781B02009A0B43138070477E
:105F600010B50C000A88023105F0AEFB208810BD88
:105F700070B504000D0004981100012B01D8042015
:105F800070BD167852781202324302800200F1325C
:105F900055701470E125002C00D10C35023B9AB2EB
:105FA0004280AA42EBD80231043005F08DFB00207C
:105FB000E6E70420009983420AD1537810781B0247
:105FC00003430B80D37890781B02034300204B805F
:105FD000704710B50C000A88023105F075FB208867
:105FE00010BD000070B501211E000420049C0E406D
:105FF0000B4218D1CB40DDB28D4214D90A49DBB235
:10600000098899420FD32300EE331D7033005800E6
:1060100011184978165C0902314301332152D9B273
:106020008D42F4D8002070BDA842FF1F10B50C00AF
:106030000A88023105F048FB208810BD10B50C78A5
:106040008B7804315C43E4B203702200013005F028
:106050003BFB601C10BD10B511000298032B01D84A
:10606000042010BD14785278043B120222430280AF
:10607000CA788C781202224342809AB28280EB2A3C
:10608000EED80431063005F01FFB0020E9E710B51B
:106090000C000B8803700B881B0A43704B888370BD
:1060A0004B881B0AC3708A880430063105F00CFB4C
:1060B000A088043080B210BD0420012B03D1002041
:1060C0001378009A1370704710B50C000B8803709A
:1060D0000B881B0A43704A880230043105F0F4FA39
:1060E0006088023080B210BDF0B589B003931E4BBA
:1060F000029242000700D05A019102F020F81325C5
:10610000061E2DD0029B01240370019B002B04D09E
:10611000001903999847001984B26B461B7A5BB249
:10612000002B0FDA1021380002F01CFB1925002883
:1061300013D130003219E1B202F066FC051E0CD119
:106140000C34A4B2042304AA380005A9938006964F
:10615000948101F0AFFD051E02D0300005F0CCFAAD
:10616000280009B0F0BDC0463464FF1F70B50500BB
:106170000C0000280CD00020814209D01022200001
:10618000044905F0A1FA01202B7823736B7863731F
:1061900070BDC0460CBB0011F0B506000D00170025
:1061A0001C0085B002291BD00020102907D1022B2A
:1061B00007D0102B03D115E00020102C08D005B01B
:1061C000F0BD69463800FFF7D1FF2A0069460BE0B1
:1061D00069463000FFF7CAFF22006946380004E034
:1061E000022BE9D12A003900300005F0DDF8E6E79E
:1061F000031CF02800D9F023032008499AB2013A81
:106200000B80D317034006499B189B100B80D30FBC
:1062100004499B185B100B807047C046AC42FF1FBF
:10622000AA42FF1FA842FF1F034B1B888B4202D3C9
:10623000024B4000C1527047AC42FF1F3464FF1F45
:10624000014B4000185A70473464FF1F1722014B5E
:106250001A8070473464FF1F70B505000E2005F0EA
:1062600033FB041E13D0D023037000230622837057
:1062700007494570033005F027FA064B2100DA8AFA
:1062800062811B7E2373044B187805F0ADF870BD56
:106290005064FF1F4064FF1FFC42FF1F262803D8E5
:1062A000024B4000C05A70470148FCE7AE42FF1F56
:1062B000FFFF000070B506000C00094D1C220021F4
:1062C000280005F051FA074B1E70074B1C7005F0B3
:1062D000ABFA0123002801D0002312202B7070BDDF
:1062E0004064FF1FFC42FF1F6164FF1F70B5050083
:1062F0000D4C0800E260A16010220021656005F0ED
:1063000043FA012803D11021A06802F058FD1022A1
:106310000021280005F038FA012803D11021606817
:1063200002F04DFD70BDC0464064FF1F70B5041EF5
:1063300005D1002903D006220D4805F0C5F90D4B03
:106340001D78012D11D1002C05D102221A7005F003
:106350003BF9280070BD00221A70074B1B78FF2BF9
:10636000F7D02000FFF778FFF3E70025F1E7C046FC
:106370005064FF1F4064FF1FFC42FF1F030010B565
:10638000002801D1002010BD00780B4A002803D15D
:106390005988D1821B7913761378022BF2D100230E
:1063A000984200D103331370044B1B78FF2B01D0AC
:1063B000FFF752FF0120E6E74064FF1FFC42FF1F8A
:1063C000002911D000280CD04B79012803D140229C
:1063D0005242134303E03F221340032802D001201E
:1063E0004B7170474022F4E70800FAE770B5094D99
:1063F0000100287800280BD0074C0622200005F069
:1064000063F921002878FFF7DBFF200005F0A4FAEC
:1064100070BDC0466064FF1F3A64FF1F00290AD0A8
:10642000012808D13F224B799343C02B03D0403B36
:106430005A425341981C704770B5174D06002B788F
:10644000FF2B15D00A2005F03FFA041E10D0D023F0
:106450000370C83B8370114B11491B784670C370A1
:106460000622043005F030F92100287804F0BCFF42
:106470000C4B1B78012B0DD10B4B1B68002B03D051
:106480009B68002B00D09847084B04211878084AD5
:1064900004F092FF70BDC046FC42FF1F6064FF1F06
:1064A0003A64FF1F5C64FF1F8864FF1F8C64FF1F3A
:1064B00060EA0000014B98687047C0464064FF1FC7
:1064C000014BDB68186870474064FF1F074B10B52D
:1064D000DA68136801331360054B1878FF2803D07E
:1064E0008021C90104F020FF10BDC0464064FF1F99
:1064F000FC42FF1FF7B50E0002F0C8F8051E1CD0C5
:106500000E4B06621F78002F00D10778AB79102060
:10651000019305F0D9F9041E0FD0D0230380C73BA7
:106520008370019BE91DC3700622043005F0CCF88E
:1065300021003800E66004F057FFF7BDFA42FF1F64
:10654000014B18787047C0466064FF1F054B002858
:1065500005D1054B1A78054B002A00D1014B1800D4
:106560007047C0465064FF1F6064FF1F3A64FF1FFE
:10657000014B58687047C0464064FF1F024B1868C3
:10658000431E9841C0B270476464FF1F421E03005F
:106590000120152A03D9FF3B5A425341D8B2704714
:1065A000F0B51C0000230E0085B0039002920B7022
:1065B000029A934201D3002019E0E55C5A1CD2B242
:1065C000002DF8D0029851198142F4DC0233DFB279
:1065D000A35C18000193FFF7D9FF002807D0013D05
:1065E000019A0399EBB233708A4202D1E01905B0E7
:1065F000F0BDDB19DBB2DBE710B50C0002F09EF852
:1066000003001220002B03D02100588805F01CF84D
:1066100010BD000070B50E4D84006359002B15D0DD
:10662000186A002801D005F07FF92B59586A002814
:1066300001D005F079F92B59986A002801D005F0AE
:1066400073F9285905F070F900232B5170BDC0462D
:106650007064FF1F1C4B70B504000E0015009942BA
:106660000AD11A4B1B68002B01D1122070BD1B6888
:10667000002BFAD09847F9E7154B994215D1134BE7
:106680001B68002B0AD01B68002B07D098470028F6
:1066900004D1104B1C70104B1D70E7E7290020003F
:1066A000FFF7AAFF0028E1D1F3E7080001F0EEFFB1
:1066B0000028DAD003780320A342D7D12900300084
:1066C00004F0C2FFD2E7C046FEFF00006C64FF1F6B
:1066D000FFFF00006964FF1F6864FF1FF7B5040037
:1066E000808801F0D3FF0025A84203D00578A08858
:1066F00002F008F81C4E3378002B1FD0AB421DD19E
:106700001A4B28001978FFF777FF002818D00023CC
:106710003370A3790820A778A688019305F0D4F8F0
:10672000011E0DD0D0230370CA3B8370019B4770BC
:1067300086808371280004F057FE01E0002DE8D127
:10674000A0880B4B8200D358002B01D0FFF762FFCB
:106750001721A088FFF768FDA08801F027FDA08819
:1067600001F0FEFDF7BDC0466964FF1F6864FF1FAE
:106770007064FF1FF0B587B01D000CAB1B880700CD
:1067800001930DAB1B88142002930EAB1B881600DF
:1067900003930FAB1B880091049310AB1B880593E8
:1067A00005F092F8041E1AD0D0230370CB3B47703B
:1067B0008370C670062229000430002D11D004F029
:1067C00083FF019B21006381029B0098A381039BAF
:1067D000E381049B2382059BA37404F005FE07B0AC
:1067E000F0BD04F0C1FFECE7F7B5009308AB1B88E0
:1067F00007000C200D001600019305F065F8041E3B
:1068000013D0280001F042FF00280FD00078D023D9
:106810002370C93BA370009B21002381019B6770FB
:10682000A580E680638104F0DFFDF7BD014B187899
:10683000EDE7C046FC42FF1F13B5040064890389DD
:10684000C2888188C0780094FFF7CEFF13BD000096
:1068500010B5044C2068002803D005F065F800232B
:10686000236010BD7464FF1FA122F0B581889200DF
:106870004A43384B384F1B6804009B189D229200F6
:106880009B18827989B01A603B68002B5FD01D7815
:10689000324B1B68002B04D05B68002B01D000201A
:1068A0009847260008363100E079FFF7B7FD237DD1
:1068B000E0710200E0780493638A29000393238A3D
:1068C0000293E3890193A38800933300FFF752FFFB
:1068D000E378002B0BD1E289A379A188029201967B
:1068E000E27928000092012201F0DAFEE0703B68B4
:1068F000002B20D0FFF7ACFF194D287800281AD0C4
:10690000184B1978FFF778FE002814D02B78E6781A
:1069100008200793A78804F0D7FF011E09D0D023D1
:106920000370CA3B4670837087808671079804F0B5
:106930005BFD00232B701721A088FFF775FCA08852
:1069400001F034FCA08801F00BFD09B0F0BD064B4E
:106950009DE7C0463409FF1F7464FF1F8864FF1F52
:106960006964FF1F6864FF1FFC42FF1FF8B5070042
:1069700008000E0001F08AFE041E18D02620FFF742
:106980008DFC051E00D12578062004F09DFF041E15
:106990000DD00021062204F0E7FED0232370C23B75
:1069A00021006770A370A680E8B204F01DFDF8BD59
:1069B000F0B585B001930AAB1B78070002930BABCF
:1069C0001B7808000D000092039301F05FFE061E85
:1069D00022D0102004F078FF041E1DD010220021C8
:1069E00004F0C2FE2620FFF759FC002800D13078C1
:1069F000D0232370C13BA370009B21002372019B15
:106A000067706372029BA580A372039BC0B2E3729E
:106A10000C9BE36004F0E8FC05B0F0BDF7B50D0099
:106A2000019001F033FE071E20D00E2004F04CFF31
:106A3000041E1BD02620FFF731FC061E00D13E7835
:106A4000D0232380C53B0622A370F91DE01C04F06F
:106A50003BFE019B2A0063810123DD401A401D405B
:106A6000210022736573F0B204F0BEFCF7BD000094
:106A7000F0B585B0029010000D0017000A9E039338
:106A800001F004FE041E31D0029B002B2ED1039B8B
:106A900002795B0724D5122313430422002E08D168
:106AA0000B99002905D10C99002902D10D990029D3
:106AB0001AD01A430D9B2271002B00D0C9E0002E82
:106AC00000D1CFE0002D00D0CCE0606A002801D0DA
:106AD00004F02AFF1C21300004F0E6FE606205E0AD
:106AE00002239A430E33D7E793432371654BBA00D1
:106AF000D458002C00D1AAE0002E10D0236A002B1D
:106B000003D11C2004F0D8FC20625E4BBA00D3589D
:106B1000186A002803D01C22310004F0D5FD0C9B1C
:106B2000002B12D0574CBB001D596B6A002B03D1B0
:106B3000162004F0C1FC6862BB00E358586A0028C4
:106B400003D016220C9904F0BFFD0D9B002B11D031
:106B50004C4DBC006659B36A002B03D1142004F0DD
:106B6000ABFCB0622B59986A002803D014220D990F
:106B700004F0AAFD380001F089FD051E67D0414BE5
:106B8000BA00D358002B62D01A6A3420002A00D1F0
:106B90001C389A6A002A01D0143080B20B9A002A5D
:106BA00001D01C3080B25B6A002B01D0163080B25D
:106BB00004F08AFE041E4AD01822002104F0D4FDFD
:106BC0002620FFF76BFB0190002801D12B78019361
:106BD000D0232370029B200063700A23294EA370E8
:106BE000039BBD00A371AB59A780196A1830002917
:106BF00005D01C22A06004F067FD200034307359DA
:106C0000996A002907D0030014221433E06002932C
:106C100004F05AFD02980B9B002B08D003001C22A5
:106C20001C330B992061029304F04EFD02987359B6
:106C3000596A002903D01622606104F045FD6B46B5
:106C40002100187904F0D0FB3800FFF7E3FC05B011
:106C5000F0BD10220D9B0D991B69A018236204F052
:106C600033FD2CE70B9B002B00D13FE7012D00D01B
:106C70003CE7606A002801D004F056FE1C210B9806
:106C80002AE7C0467064FF1F10B5044C2068002836
:106C900003D004F049FE0023236010BD6464FF1F8D
:106CA0000B4B07B51A68002A01D100200EBD6946BA
:106CB000531C012012780731FFF772FC0028F4D032
:106CC00002780123100018401A42EED0EEE7C046C9
:106CD0008064FF1FF0B51F4F01203B6887B0002B79
:106CE00025D09B78059300F0B3FB002821D00A2023
:106CF000FFF7D4FA04000B20FFF7D0FA164B05007B
:106D00001E78731E9E413B68F6B2191DD878FFF7B6
:106D100057FB3B682900DA7A043303929A7901938E
:106D20000292009033002000059A04F0EDFB07B0BA
:106D3000F0BDFFF7B5FF002805D00620FFF7AEFA3B
:106D400004000720D8E70820FFF7A8FA040009206C
:106D5000D2E7C0466464FF1F6064FF1F70B50A4E2F
:106D6000040033780D00FF2B0DD0042004F0ACFD9F
:106D7000011E08D0D0230370CE3B45708370C470D1
:106D8000307804F031FB70BD0C43FF1F70B5040078
:106D900006200D0004F098FD011E0AD0D0230370D8
:106DA000CD3B8370054B44701B688580187804F0D8
:106DB0001BFB002C01D0FFF767FF70BD6464FF1F51
:106DC000F8B5264F06003B680D001124002B05D1B5
:106DD0000522234B1B78134202D112242000F8BD58
:106DE000204A10241268002AF8D01278002AF5D020
:106DF000DB0719D52B789A1E012A1AD80C2004F02B
:106E00005BFB132438600028E8D000230A2243707B
:106E100029000670023004F057FCFFF75BFF041EE8
:106E20000AD0FFF731FFD9E700F012FB0028E1D1CB
:106E3000E4E7002BE2D0D0E70B4B1B78032BCDD13E
:106E40001D20FFF72BFA094B18800028C6D0084BED
:106E500004211878074A04F0AFFABFE76464FF1F03
:106E60006164FF1F8064FF1F6064FF1F5E64FF1F7B
:106E70008C64FF1F60EA0000F7B50193194B140002
:106E80001A78052306000F0012201A4221D001298A
:106E900020D1154B1D68002D1BD002201F2C18D8A7
:106EA000002C02D0019B002B13D0104B1F221E7010
:106EB0006E1C0021300004F057FC019922003000C4
:106EC00004F002FC310020002C70002F06D004F0EA
:106ED00013FDFEBD064B12201D68DCE704F014FC18
:106EE000F7E7C0466164FF1F8064FF1F0C43FF1F6C
:106EF0007C64FF1FF8B50F4E12243368002B17D0A7
:106F00001B780F3C834213D100250B4F02213878A8
:106F100004F07AFB094B042138781D8004F074FBDF
:106F2000074B28001D8033685C7004F005FA0400EC
:106F30002000F8BD6464FF1F8C64FF1F7864FF1F8E
:106F40005E64FF1F70B5012823D11B4C2388002BE2
:106F500003D01A4A1578002D07D0194B1B68002B57
:106F600002D01878FFF7C6FF70BD3B2B02D93C3B1F
:106F70002380F9E7134E0221307804F045FBFA2212
:106F80002388920002215A43307804F0CDFA2580FC
:106F9000EAE70B4B1B68002BE6D00B4B1B785B071B
:106FA000E2D5084B0221187804F02EFB0022024B98
:106FB0001A80FFF769FED7E77864FF1F5C64FF1F44
:106FC0006464FF1F8C64FF1F6164FF1FF8B51E4DD2
:106FD0002868002803D004F0A7FC00232B601B4E78
:106FE0003068002803D004F09FFC00233360184F62
:106FF00005243B7818002040234221D0154800F09A
:107000002BFA3B78234213D0202004F055FA286055
:10701000002813D02022002104F0A6FB202004F039
:107020004BFA041E306005D02022002104F09CFBA6
:10703000002004E0286804F077FC2C601320F8BDE1
:1070400000F00AFAF4E7C0468064FF1F7C64FF1F6B
:107050006164FF1F0043FF1F10B50A4C23681A1E0E
:107060000ED0002808D10130587004F065F90028CE
:1070700005D02368002B02D00021FFF787FE0122F4
:10708000100010BD6464FF1FF7B5274E050033687C
:107090000191181E21D05C78244F012C30D1FFF7CC
:1070A000FFFD002825D02000FFF7F8F80400412854
:1070B00014D91F4B022118781E4A04F07DF91E4B8B
:1070C0003C3C1C80022233685A703B78002B14D160
:1070D00028000199FFF75AFE0120FEBDFA22920016
:1070E0004243002AEED0124B0221187804F01CFA19
:1070F000E8E7FFF7D3F80200F3E700233B70EBE784
:107100003B78002BE8D1032004F0DEFB011E08D001
:10711000D0230370CC3B457083703368187804F03B
:1071200063F9FFF7B1FDD7E76464FF1F5C64FF1FDD
:107130008C64FF1F60EA00007864FF1F10B51749D8
:10714000838802008B4220D011D815498B4217D07A
:10715000144900205B1899B2012907D89268117868
:107160005A425341D8B2FFF7F9FD012010BD0E4A33
:1071700000209B1807229BB29A424041C0B2F5E71B
:1071800083681878FFF768FFF0E7836899785A7882
:10719000090218781143FFF777FFE7E70A2000009C
:1071A00006200000F8DFFFFFAFDFFFFF014B187084
:1071B0007047C0460D43FF1F10B5064C207001F00C
:1071C00041FA207804F090F90521207800F062FD62
:1071D00010BDC0468C64FF1F0BB273B50D00002BB1
:1071E00000DBC4E0884B187804F0AEFB041E0ED020
:1071F0000378912B0FD0A22B00D1A1E0834B1878FC
:10720000FF2852D0210004F0EFF800284DD1802053
:107210000002684076BD43780F2B76D013D8052B3B
:1072200070D00E2BEAD18088794B98422BD8794BBD
:1072300098421BD8784B9842E0D1A3681878591C23
:10724000FFF774F838E03E2BD8D18378032B74D045
:107250006CD8012B6ED0022BD0D1704B1B68002B49
:1072600023D05B68002B20D098471EE06C4BC018E1
:107270000C28C3D804F010FB1DC2C2150BC20B0BA7
:107280000B3223C23C00674BC0180728B6D8664BA8
:107290001B68002B09D01B68002B06D020009847E4
:1072A0000AE0A3681878FFF7C7F8200004F01CFA7A
:1072B000ADE7A068FFF762F800289FD0F5E7A36864
:1072C0001B78002BF1D0554B1B68002BEDD01B68B1
:1072D000002BEAD0210055489847EDE74F4B1B683B
:1072E000002BE2D01B68002BDFD021005048F3E7D1
:1072F000504B1B68002BD8D05B68002BD5D02100E9
:107300004348E9E7FFF7EAF9CFE780884A4B98421C
:1073100003D04A4B984200D070E7464B1B68002BC5
:10732000C3D05B68002BC0D02100D5E7153B012BF3
:10733000BBD963E7FFF798FAB7E7FFF77DFAB4E741
:107340003F4B1B78042B07D100236A461380017939
:10735000408800F0C5FCA8E7364B1B68002BA4D082
:107360005B68002BA1D00100364898479DE70124B7
:1073700021420AD0294B1B68002B04D05B68002BEC
:1073800001D000209847012043E78B070AD5264B00
:107390001B68002B04D05B68002B01D020009847AD
:1073A000022036E70421280008400D4200D131E7D1
:1073B000254E3388002B21D0013B9BB23380002B1C
:1073C0001AD1FFF7DBF800280AD0204B1C70164BAF
:1073D0001B68002B04D05B68002B01D0200098476D
:1073E000FFF7C6F8694601F001FD6846FEF7FEFFAB
:1073F0001D20FEF753FF308004200AE7024B187867
:1074000004F002F9F8E7C0468C64FF1F0D43FF1F2C
:107410000E20000001200000091000008464FF1FFE
:10742000FEDFFFFFAFDFFFFF8864FF1F0C200000BF
:107430000B2000006C64FF1F0D20000013200000D3
:107440006164FF1FFFFF00005E64FF1F5C64FF1F9D
:1074500010B501F09BF910BD014B18607047C04694
:107460008864FF1F0B880020162B01D817230420E7
:10747000014A13807047C0463664FF1F00207047E2
:10748000074A03001188814207D091880020994261
:1074900002D101308000101870470020FAE7C04682
:1074A0009464FF1FF0B58F7806000D00C5B01E2F45
:1074B00015D1FFF7E5FF051E03D10024200045B0DC
:1074C000F0BD00223B003100C078009200F0B2FB1A
:1074D0000400A81C00F0D2FBFF23EB70EEE7264B64
:1074E000062403931B78FF2BE8D0182FE6D87B08DF
:1074F000224A013BDB0002929A589446002ADDD0D2
:10750000029AD3185B68002BD8D00878002802D1E3
:107510004B78012B02D10624122FCFD107AFAB88B5
:10752000697800976446AA68A047041EC6D1AB7864
:10753000029A5B08013BDB00D318390030005B681E
:107540009847041E0BD1AB78042BB6D0039A3100B8
:1075500010782200009700F06DFB0400AEE76A7817
:10756000002AABD1AA7805A93B88087130000A70BF
:107570004B80FEF747FBA0E71043FF1F1CBB001129
:107580001D4B37B5050098420BD000290AD1FFF7F3
:1075900077FF002805D11948FFF772FF002800D0B7
:1075A000058037BD01291AD1FFF76AFF041EF8D004
:1075B00001235B420380A378FF2BF2D0FE2B07D080
:1075C0000023E0781422009329001E3300F032FBE0
:1075D000A01C00F053FB01235B426380E1E702291A
:1075E000DFD1013901F0BEF80028DAD12800FFF719
:1075F00047FF041EDFD1D4E7FEFF0000FFFF0000BD
:10760000022210B5074B52421A80074801325A80B5
:107610009A80DA8000F07EFA044801F025F8002014
:1076200010BDC0469464FF1FA57400118175001140
:107630000388F7B50400002B02D102252800FEBD07
:1076400042680221137825485268FEF7A5FD0028FC
:107650002ED0234F01253A88002AEFD0802321889D
:107660005B0201259B1A9942E8DC0C2003F024FF01
:10767000061E31D03B8822889C46002318000195C5
:1076800061469DB2491989B2AA421BD8002801D08F
:1076900062443A8000233000082208C0210004F030
:1076A00013F8104A1368002B13D100251660C5E7A4
:1076B0006268022113780C485268FEF76DFD0028BD
:1076C000C7D1BAE760681D014019418101330198B3
:1076D000D6E71A001B68E6E71325AFE78ABB00115F
:1076E0000E43FF1F9064FF1F88BB0011014B1870F1
:1076F0007047C0461043FF1F14230A0010B51A40FC
:10770000194204D00122102101F048F810BD4B06A7
:10771000F9D4012088434000F8E710B514008B0627
:1077200004D50122102101F039F810BD08230A0008
:107730001A40194202D14BB2002B0FDA102101F08E
:107740002DF8002808D02300F2331B78002BECD052
:10775000F1342378012BE8D10020E6E703208907E4
:10776000FAD4E2E7F0B51F00184B85B01C68019011
:1077700002910392002C27D1200005B0F0BDA5682E
:107780003301ED186B89019A934211D3029A934207
:107790000ED8002F04D10A9B002B10D12C00EBE750
:1077A0003B002978039A6868FEF7F6FC0028F2D1BE
:1077B0000136B6B2A388B342E1D82468DAE7A368F9
:1077C0000A9A5B891380E9E70026F3E79064FF1FBC
:1077D00037B50C000A8849880123914217D3002A43
:1077E00015D0651D23792A0002210A48FEF7D4FC32
:1077F000102300280BD023796188208800242A00D8
:107800000094FFF7AFFF0A23A04200D02300180026
:107810003EBDC0468ABB001113B50A0008884988DE
:10782000012388420BD8002809D00024137905329F
:107830000094FFF797FF0A23A04200D0230018000E
:1078400016BD13B50A0008884988012388420BD861
:10785000002809D00024137905320094FFF782FF35
:107860000A23A04200D02300180016BDF0B58BB04B
:1078700003904A8808880E000123824255D30028CD
:1078800053D00023012704AC237000227188130019
:107890000092FFF767FF051E3ED02078002835D103
:1078A0002B78022B18D167706A8983000130E318A6
:1078B00080005A8069680222201803F005FF2378AF
:1078C0000133DBB22370042B19D93B0068890130E6
:1078D00080B2002BD9D01FE00223637012235843DB
:1078E0006A89231804305A8069681022201803F02E
:1078F000EBFE23780133DBB22370002BE5D10C4A79
:107900006B899B185A425341DBB2DFE76378012B46
:10791000E4D12B78022BC7D022780A23002A04D086
:1079200021000398FEF798F9002318000BB0F0BD72
:107930000100FFFF0F4BF0B504001868002816D0B7
:1079400083685D89A54207D88288AE18B44203DAFD
:1079500012019A18934201D10068EFE71E005F8977
:107960001036A74204D1002900D00D801800F0BDC8
:107970003300EFE79064FF1F70B505000C00088826
:107980000021FFF7D7FF03000120002B04D02200C5
:107990002800197AFFF7C1FE70BDF7B50C0000256D
:1079A00001902300EE331B78AB4201D800200AE09F
:1079B0006B00E65A00213000E718FFF7BBFF0028F4
:1079C00002D126800130FEBD017A0198FFF794FEB6
:1079D000002802D03B882380F5E70135EDB2E0E7CF
:1079E00010B5040008880021FFF7A4FF0300012060
:1079F000002B03D02000197AFFF77EFE10BD000097
:107A0000054B1B68002B01D1180004E09A685289CD
:107A10008242F6D1988870479064FF1FF0B50E2718
:107A2000002687B0039302ABFF183E8005001F4B72
:107A300040891400984207D02B78013000976A687B
:107A400080B2FFF78FFE060002212B7818486A6883
:107A5000FEF7A2FB00280FD06C892000FFF7D0FFB3
:107A6000002802D0013C0419A4B2039B002B00D0D3
:107A70001C80300007B0F0BD02212B780D486A68E9
:107A8000FEF78AFB0028E7D102212B780A486A68B2
:107A9000FEF782FB002807D0002EDED03B88A342F1
:107AA000DBD17489013CDFE76C89DEE7FFFF000072
:107AB0008ABB001188BB001186BB001110B50C00F9
:107AC000FFF7DEFC03000220002B0AD0002C00D0C0
:107AD00023609B781720FE2B03D00138FF2B00D1A9
:107AE000002010BD73B50D0001A904001600FFF7BA
:107AF000E5FF172805D0002E04D129002000FEF74D
:107B000027F976BD01221021200000F047FE002851
:107B1000F3D0F6E7014B18607047C046A064FF1F22
:107B200037B56B469D1D010004000222280003F0BA
:107B300003FF2B88B02B0ED12379122B09D1230000
:107B4000FA331B78012B06D10121608800F0E0F8A0
:107B500001E01B2BF8D037BD10B5054B0421187080
:107B600000F098F8FFF74CFDFEF770FB10BDC04623
:107B7000A464FF1F0020F0B50BB20F0087B0834252
:107B800034DA274B187803F0DFFE051E2BD003787C
:107B9000A02B25D103AE3100FEF7E4F8041E0BD173
:107BA000B378DB0724D51F4B06341B68002B03D0AA
:107BB0003100688898470400A868002801D003F0C5
:107BC0009BFD002C08D1184A039B1340174A93428F
:107BD00006D0B3781B2B03D00121688800F098F8F9
:107BE000280003F081FD80200002784007B0F0BD3E
:107BF0000F4B1B68002B10D0310068889847041E7B
:107C0000DAD07378002BD7D1B27801A90A704B80F3
:107C10000C716888FDF7F6FFCEE70624F1E7C04651
:107C2000A464FF1F9C64FF1F00FFFF0000011200FF
:107C3000A064FF1FF7B50190FC200D0017001E0087
:107C400003F042FE04001320002C12D0B0232000C9
:107C50002370089BF4226770658026710830002B22
:107C600008D0190003F030FD2100019803F0BCFB9F
:107C70000020FEBD089903F077FDF5E710B5041E5E
:107C800006D00078FD2803D803F086FCFF2323707C
:107C900010BD00000A1F93B210B504000220032B90
:107CA00005D882400020024BD1529B189C7010BD19
:107CB000C464FF1F0B8870B5043B04000D00022054
:107CC000032B0BD80121200000F04CFD03001420F1
:107CD000002B03D02900200000F0DEFB70BD000067
:107CE00007B51300034A00920A00012100F02CFCA2
:107CF0000EBDC0461D7F001107B501920322009200
:107D0000024B0A00122100F049FC0EBD9B7F0011BE
:107D100007B56B4601AA11800449D880087806335C
:107D2000012802D1190003F03FFD07BDA564FF1F24
:107D30000C4B10B518700023FF210B4A13801381E0
:107D400093819380094A5380137051729381937287
:107D5000D174D3821375517703F00EFB00F0FCF958
:107D600010BDC046D464FF1FC464FF1FA664FF1F7C
:107D7000F0B58DB06B46002003910C229B5E8342D0
:107D800000DBB0E05D4B187803F0DEFD051E00D18E
:107D9000A4E00378902B00D09DE006AF0100468858
:107DA000380000F013FA79680400002900D19CE043
:107DB0003B88052B6ED13B89032B1CD905AC2000D9
:107DC00000F0A2F86288172A61D83989131D9942F8
:107DD00031D17968237804310291D90738D5607898
:107DE00000F08EF9071E06D0002303712378012BC3
:107DF00008D0132B23D0A868002800D178E003F026
:107E00007BFC75E06288029909A800F0A6F8029050
:107E1000380000F08BF909AA2378387A0192002201
:107E200031000092029A00F012F9380000F064F973
:107E3000029B002BDFD0300000F080F9DBE70378F5
:107E4000032BD8D16288029909A800F0D6F8DEE7A2
:107E5000122B13D1029909A800F0B5F8021EEAD13D
:107E600027498B88002BC6D0887909A923780191EE
:107E700061780091310000F0EAF8BCE7002302AA23
:107E800093833000617809AAFFF72AFFB3E71D4BFF
:107E90000993F6E7042B02D09A1F012AABD8184A9F
:107EA000043B9B00995A0029A5D0D2189078310044
:107EB0003A0000F0AEF800289DD13B88042B03D097
:107EC00001213000FFF724FF012C04D1A86800280D
:107ED00001D003F011FC280003F006FC8020039B76
:107EE0000002434018000DB0F0BD012800D182E728
:107EF00001213000FFF70CFFEDE7C046D464FF1FFF
:107F0000C464FF1F010017000B7803704B784370A7
:107F1000CB788A781B021343438070470A8803009A
:107F200002700A88120A42700A88012A06D14A8819
:107F300082704A88120AC27004207047022082426E
:107F4000FBD14A8804309A704A88120ADA708A880B
:107F50001A718A88120A5A71EFE710B504000120DD
:107F600082420CD94B780A781B0213432380834248
:107F700006D1CB788A781B0213436380002010BDA2
:107F8000022BFBD1CB788A781B02134363804B7999
:107F90000A791B021343A380F0E70B8803700B8858
:107FA0001B0A43704B8883704B881B0AC3708B88F5
:107FB00003718B881B0A4371CB888371CB881B0AA2
:107FC000C3710820704703000120082A14D14A78A1
:107FD0000878120202431A80CA7888781202024393
:107FE0005A804A790879120202439A80CA798879BC
:107FF000120202430020DA80704710B5040001200D
:10800000022A05D100204B780A781B0213432380F3
:1080100010BDF8B5060010200F00150003F054FC49
:1080200004000120002C0ED0A0230C222900238064
:108030006780201D002D07D003F046FB2100300093
:1080400003F0D2F90020F8BD03F08EFBF6E7F7B598
:108050001E00009008AB142017001D78019103F05A
:1080600033FC041E12D0A2230370019B477043808F
:10807000099B057146710C220830002B07D01900AE
:1080800003F022FB2100009803F0AEF9F7BD099937
:1080900003F06AFBF6E737B5041E0FD04388002BC8
:1080A0000CD00025C1881323007A17220195009572
:1080B000FFF7CDFFFF2365806372257037BD000099
:1080C00010B50C4904004A88002A09D08B89002B7E
:1080D00005D00020CB8A0222834201D010BD0122AC
:1080E00013000A20434300204032C854C81842807D
:1080F0000472F3E7A664FF1F0023438003707047F8
:10810000094B00211A0010B55C88002C06D01C79A0
:10811000844203D10A234B43D01810BD01310A33E6
:108120000329F1D10020F8E7A664FF1F10B5040071
:10813000407A03F031FAFF23637210BD70470430B8
:1081400010B580B203F068F9002803D00421494239
:1081500003F002FA10BD000070B50025104CA068B5
:108160002580A581A580A84202D003F0C5FAA560AC
:1081700000250C4C0C4B606D1D80230058331D7086
:10818000A84202D003F0B8FA6565002560680028AF
:1081900001D003F0B1FA013508340A2DF6D170BDD3
:1081A0006C65FF1F1065FF1F6065FF1F70B5041E23
:1081B00009D1054D2880A881A880A868002802D090
:1081C00003F09AFAAC6070BD6C65FF1FF0B54B8888
:1081D00085B00193002343600A7905000F00022A4D
:1081E00000D07BE0CA88032A17D98B685E7819789B
:1081F0003602DC78D8790E4399781B7A24021B0268
:108200000C43034353495BBA0B80331D93421ED189
:10821000042C04D0631F022B0ED9012015E0019A13
:108220004D4B1201D35A002B06D00198FFF7BEFF29
:108230004A4A1369013313610421B8682E812C80E6
:10824000494203F089F96860002005B0F0BD434D54
:10825000042C06D0631F022B0FD9EB680133EB60AF
:10826000DBE7019A3C4B1201D35A002B05D0019851
:10827000FFF79CFF2B6901332B61374B30000293D2
:10828000019B029A1B010193002301998C468B529A
:10829000130063449C8003939E81FFF750FF039B70
:1082A000041E986016D00421B868494203F054F9BE
:1082B000FA880100043A200003F006FA0199029AB4
:1082C000FB888A5A043B9B18029A8B522B68013315
:1082D0002B60A2E7AB690133AB619EE71E4B0293B3
:1082E000019B1E01029BF35A002B2DD002998C1981
:1082F000A068002828D0012A26D1FA889B189BB2B2
:108300007352A189994217D39B1AC018B96803F018
:10831000DBF9029BA289F35A934200D07DE7002249
:108320002B81A3882B80A3686B60029BF2520B4ABF
:1083300053680133536070E7084A936801339360D0
:108340000198FFF733FF68E7044A5369013353612B
:10835000F6E7C046D664FF1F6C65FF1FDC64FF1F95
:1083600070B5051E15D10B4C0B4B188023005833EC
:108370001870606D002802D003F0BEF96565250015
:1083800050356068002801D003F0B6F90834AC42DB
:10839000F7D170BD1065FF1F6065FF1FF0B51700B6
:1083A000A12285B0920001934243394B06001B681D
:1083B0000C009B18D933FF331D78FDF741FF0430C3
:1083C000854204DD3000FDF73BFF0430C5B2BD42FD
:1083D00007D33A0000213000019B03F09DF905B05E
:1083E000F0BD2900380003F047FA2300C6B250332D
:1083F0001E700393019B29006365380003F0F4F9B4
:10840000CBB20293002B02D0039B01361E700026D4
:108410002300503303931B78B34204D8606D0028C7
:1084200031D10020DBE7029A2800002A04D0013B6A
:108430001000B34200D02800F700E719387003F0AD
:108440006BFA786000280ED03A78019903F03CF975
:10845000019A3B780136D3180E4A0193D369F6B2DC
:108460000133D361D4E7039B18706065A74205D13F
:10847000084A1320D36A0133D362B0E7606803F07F
:108480003BF90834F2E703F037F900236365C8E7E6
:108490003409FF1FDC64FF1FF7B50D00070004213E
:1084A000686803F059F82B89040003702B891B0AB4
:1084B00043702B8883702B881B0AC3702E8902257A
:1084C0000436F6B2F42E15D81B4B9F4214D10C2063
:1084D00003F0FAF91135011E0CD0902303708E3B86
:1084E0000371043B4380154B8460C680187802F00A
:1084F0007BFF00252800FEBD5C237B43104AD31878
:108500000093583301931B78002B0FD103003200E6
:1085100038000099FFF742FF019B05001B78002BF4
:10852000E8D13800009903F0C7F8E3E7054A0725CA
:10853000536A01335362DDE7FEFF0000D464FF1F7E
:108540001065FF1FDC64FF1FF0B587B00090172097
:108550000F0016000193FFF7F2FD1325041E19D03A
:108560000C98031E02D00199201D9847030AE3705E
:10857000052302AAA07004309081277000986670CD
:1085800003A993800494FFF787FF051E02D0200003
:1085900003F0B2F8280007B0F0BD0000F0B587B0D6
:1085A0001F000CAB1B780391059301210DAB060056
:1085B0001C78049200F0D6F81425002821D0200061
:1085C000FFF77EFD0135041E1BD01149059B0A787B
:1085D00003700132D2B2131EC68001D101231A00EA
:1085E0000B7022713000049B03990097FFF7ACFFDA
:1085F000051E09D1230021000648074A093302F06D
:1086000033FF280007B0F0BD002363802370F8E734
:10861000D864FF1F9780001130750000F8B5050081
:108620000E00064C064F2368002B02D031002800B4
:1086300098470434BC42F6D1F8BDC0467C65FF1FA4
:108640009065FF1F0123064A5B425380002313718C
:108650005362044A136053609360D36013617047A0
:108660009065FF1F7C65FF1F0200002310B50649BF
:108670009C000859002801D1625010BD0133052B20
:10868000F6D11320F9E7C0467C65FF1F034A5388E3
:10869000181A434258414042104070479065FF1FEE
:1086A000F0B585B002930AAB1F780CAB1B88009025
:1086B00008000E0001920393FFF7E8FF0500112068
:1086C000002D1BD10E48FFF7E1FF04001520002C00
:1086D00014D006220B99A771E01D02F0F5FF019B53
:1086E00030002371029B29006371009B6680237018
:1086F000039B6562E381FFF791FF280005B0F0BDA1
:10870000FFFF000010B5FFF7C1FF04000220002C9E
:1087100012D060880121FFF781FF606A002801D034
:1087200003F002F928220021200003F01DF80123A4
:1087300000205B426380207110BD000030B5074A05
:10874000074C5588010013780020A54204D05B1A1D
:1087500059424B415842104030BDC0469065FF1F02
:10876000FFFF0000084A10B501230C00904208D01A
:10877000FFF78CFF031E04D0037923405A1E934158
:10878000DBB2180010BDC046FEFF0000024B187996
:10879000431E9841C0B270479065FF1F70B504003A
:1087A0000D001600FFF772FF002804D10D4B9C420C
:1087B00000D0143070BD416A03790520002907D02C
:1087C00012221A40102A02D10520002EF2D10F20C9
:1087D000DB06EFD5897E0C20A942894149424942F6
:1087E0000840E7E7FEFF0000030010B5002800D1B5
:1087F00010BD0348034A41889142F9D09847F7E7F2
:108800009065FF1FFFFF0000002330B5C45CCD5C06
:108810006C40D4540133102BF8D130BD0F2300220B
:1088200010B5C45C64002243CA54C25CD209013B47
:10883000F7D210BD0200010010B52032103102F055
:1088400043FE10BDF0B58BB00390102005931700C8
:10885000049102F031FE0090102002F02DFE009BEA
:1088600013240190002B05D000280CD1132400986C
:1088700003F05AF8019B002B02D0180003F054F8C3
:1088800020000BB0F0BD102002F016FE06001020F4
:1088900002F012FE13240500002E00D1AEE00028E5
:1088A00019D01022002102F05FFF32002900039846
:1088B00002F00AFE041E0ED133787F2B51D830000F
:1088C0000099FFF7ABFF009B1B787F2B53D80199D2
:1088D0000098FFF7A3FF300003F026F8002D02D028
:1088E000280003F021F8002CC1D1102002F0E4FD93
:1088F0000600102002F0E0FD0290002E7CD000283F
:1089000078D03A000F3223000125121105D00F3321
:108910003B4015B25A4253411BB26A1E1201002B52
:1089200033D0049BD2B298180099029AFFF76CFFDB
:10893000013D10220021300002F016FFADB2049F6D
:108940002D017D19AF4242D0002C33D0300002F00F
:10895000EBFF029B002B00D189E7180002F0E4FF37
:1089600085E729003000FFF759FF28002549009AC4
:10897000FFF74AFFA7E729000098FFF74FFF2800FD
:108980002049019AFFF740FFA5E70F210F40049906
:108990008A18D9B28F4208D9D15C06A8195401337C
:1089A000102BF6D1029A0199C0E7791A4842414149
:1089B000C901F2E73900300006AAFFF725FF3200AF
:1089C000039806A902F080FD10370400BAE7002CD6
:1089D000BCD13000029906AAFFF716FF320006A9A3
:1089E000039802F071FD082204003100059802F09E
:1089F0006BFEABE71324A9E71324AAE7002800D0F5
:108A00006EE733E790BB0011F0B58BB00F00160096
:108A10000225009000283FD0002A3DD00B1DDBB27C
:108A20001800029302F048FD1135041E34D0FDF702
:108A300047FD05003A000099201D02F01DFDEBB234
:108A40000393E3702B0CDBB22F0A00936370FFB229
:108A50002B0E2370A7700193FDF72CFD102201004F
:108A600006A802F009FD2100029A04AB06A8FFF750
:108A7000E9FE051E0DD1039B08223370009B04A95B
:108A8000B370019B7770F370301D02F0F5FCFDF7B9
:108A90001DFD200002F048FF28000BB0F0BDF0B52E
:108AA0008FB00D00149E039004920593002A03D109
:108AB000022420000FB0F0BD002EF9D00398FFF77C
:108AC000E5FD1424071EF4D07278337812021A439D
:108AD000B3781B041343F27812061A43036A019217
:108AE000934201D30133E3D1002D03D03B7901241C
:108AF0009B07DED50822002106A802F035FE059B63
:108B000013240433DBB21800029302F0D5FC051ED7
:108B1000CFD0059A0499043002F0AEFC0422310053
:108B2000280002F0A9FC3900102210310AA802F036
:108B3000A3FC2900029A06AB0AA8FFF783FE041ED5
:108B40000FD1082206A908A802F096FC0822311DC0
:108B500008A802F029FC012807D101990398FDF724
:108B6000C9FC280002F0E0FEA3E70124F9E70000B9
:108B700070B51C4C05002368181E10D0002D14D1B0
:108B80001A78002A0CD1981C083202F09DFD02F0E0
:108B9000FBFB0135002808D123681D70012070BD42
:108BA0000A331800082202F08FFD2368002BF5D04D
:108BB000122002F089FE061E0DD0C1232168037029
:108BC000457002311022023002F07EFD2368310030
:108BD000587802F009FC206802F0A6FE002323600A
:108BE000DCE7C046B865FF1FF8B504002020FDF79C
:108BF00055FB0D4EA700BB590500002B0DD00028DA
:108C00000BD0D878FF2809D108492A000C55F35910
:108C100007480333611802F027FCF8BD290002F071
:108C20001BFC0028F0D1F8E7D465FF1FBC65FF1FCF
:108C3000419E001170B5064D84006359002B05D08C
:108C4000D87802F0A9FCFF226359DA7070BDC046E3
:108C5000D465FF1F70B506008CB00C001500002114
:108C60003022684602F080FD31001022684602F092
:108C700003FC1D2021000322684402F0FDFB68462E
:108C8000FFF7D8FD2D21040003222800694402F0DB
:108C9000F3FB20000CB070BDF0B50700160097B0D4
:108CA00001931CAB1D7830221EAB00910AA8002155
:108CB0001C7802F059FD102239000AA802F0DCFBF2
:108CC0001022002102A802F04FFD0722310002A865
:108CD00002F0D2FB072202AB9818631E9C41019957
:108CE00002F0CAFB02AB9C732B005A1E934102AAEE
:108CF000D3730021102206A802F036FD06221D992A
:108D000007A802F0B9FB1A2002ABC01806221F996F
:108D100002F0B2FB102200990EA802F0ADFB102267
:108D200002AB0EA908781C78013A6040D2B20870F4
:108D300001330131002AF5D10AA8FFF77BFD10228B
:108D400012A904000EA802F0BFFC102206AB0EA967
:108D500008781D78013A6840D2B2087001330131B9
:108D6000002AF5D10AA8FFF765FD044310222098D8
:108D7000E4B212A902F080FB200017B0F0BD70B57C
:108D80000E0014008CB00100102268461D0002F095
:108D900073FB3100082204A802F06EFB21000822B8
:108DA00006A802F069FB6846FFF744FD04001022A4
:108DB000280008A902F060FB20000CB070BDF8B5D7
:108DC00006000D0000243719AC4200D3F8BD02F0B4
:108DD0000BFC030A3B70631CDBB201379D4203D9D5
:108DE0000234F054E4B2EEE71C00EDE773B5060080
:108DF0000C000225002819D0002917D0032101A852
:108E0000FFF7DDFF6B469A793F231A400133134386
:108E10006A463000937101A92200FFF71BFF051E6F
:108E200004D10322E01C01A902F04EFC280076BD0B
:108E300003785807DA08C00FD20080009B07104360
:108E40009B0F1843C0B2704707230B40C908C900E5
:108E50000B4303707047000070B50400FFF7EAFE93
:108E6000134DA4006359002B21D0186A002801D0AB
:108E700002F05AFD2B59986E002801D002F054FDE3
:108E80002B59D86E002801D002F04EFD2B59186FD7
:108E9000002801D002F048FD2B59586F002801D05E
:108EA00002F042FD285902F03FFD00232B5170BD16
:108EB000D465FF1F0E4B8000C35870B50C00002B0B
:108EC0000FD09D68002D0CD02B78201D0B706B7877
:108ED0004B70A97CFFF7B8FF2B7E23726B69E360B0
:108EE00070BD10220021200002F03EFCF8E7C046D1
:108EF000D465FF1F014B18607047C046D065FF1F47
:108F0000074A03008000825810B5002A06D0D08896
:108F1000984203D1012901D1FFF79EFF10BDC04641
:108F2000D465FF1FF0B5264E95B087000B93BB5953
:108F30000500099112200A92002B31D0D888FFF742
:108F4000A5FB04001420002C2AD0280010A9FFF74C
:108F5000B1FFBB591E781D6A002E23D00895FDF77E
:108F6000EFFA07000020FDF7F1FA0790A379E61D5C
:108F7000069310AD0CA9089800F0E2FA0EA928009B
:108F800000F0D7FA0B9B0A990493069B0998029369
:108F9000079B0396019300970EAB0CAAFFF77CFE8C
:108FA00015B0F0BDFDF7CCFA06903000FDF7CEFA13
:108FB000E31DA779079310AB06000893DAE7C046D4
:108FC000D465FF1F30B50C4C85002A59030085B0CD
:108FD0000120002A0ED018006946FFF76BFF2B59BD
:108FE0001A78D888054B002A00D1054B6A4607211C
:108FF00000F0D9FB05B030BDD465FF1F33950011DB
:109000004195001130B5094C8500295985B01022D1
:109010006846253102F058FB2A591121044BD088AB
:109020006A4600F0C0FB05B030BDC046D465FF1FE6
:10903000DD95001130B5094C8500295985B0102205
:109040006846353102F040FB2A591121044BD08883
:109050006A4600F0A8FB05B030BDC046D465FF1FCE
:109060001B960011F7B54D4F86001020F4590D00E6
:1090700002F022FAF3592062186A132200286CD0F9
:10908000033A29009C6802F01FFBF3591A780192F9
:10909000002A58D11E6A227D317B9446514001221C
:1090A000019F114201D167461740217D9143394309
:1090B0002175377B4F40BC4660460027800701D4AE
:1090C0004F081740012102208F40227D82433A43FE
:1090D0002275377B5740BC4660460027400701D4C5
:1090E00097080F400420227DBF0082433A43227537
:1090F000627D002794466046727B42400A4201D15D
:1091000067460F400121627D8A433A436275777B4F
:109110005740BC4660460027800701D457080F40DF
:109120000220627D7F00824317436775767B0022B1
:109130007E40760701D4BA080A400426617D920079
:10914000B1430A4362756A78002A08D06278002A1F
:1091500005D005220533DA7700221000FEBD042277
:109160002979114205D1A17C114202D10533033A7C
:10917000F1E7019A21782C78002A02D10A00210017
:10918000140018220429E8D8042CE6D805206043EE
:10919000034A05331218525CDDE7C046D465FF1F51
:1091A000A0BB001110B50A001121024B00F0FBFA20
:1091B00010BDC046779600110B0030B587B001ADE9
:1091C0002B806B4604001100981D082202F07CFAE7
:1091D0002A000B212000024B00F0E5FA07B030BD59
:1091E0009F96001110B50A001121024B00F0DBFA26
:1091F00010BDC046F396001113B50B0011006A466E
:1092000013706B4604000622581C02F05DFA6A4691
:1092100008212000014B00F0C6FA13BD139700117E
:1092200010B50A001121024B00F0BDFA10BDC04676
:10923000639700117FB505000B4BAA00D4580800B6
:10924000002C0FD0666F237FE28821780396266F6B
:109250000296E66E0196A46E0094FDF709FC2800C4
:10926000FFF7FAFD7FBDC046D465FF1F10B517217B
:10927000FFF7E0FF10BD000070B50A000D00064BBF
:109280000221040000F08FFA060029782000FFF781
:10929000D1FF300070BDC0464396001170B586B056
:1092A00000236A461370836804001D78681E0A282C
:1092B00059D801A902F0A0FA060633373B3F4347CD
:1092C0004B4F5300180000F042F9062312284BD0F0
:1092D00000281BD16088FFF7D9F90823002813D094
:1092E0004279002A47D1264B1A78072312070BD55B
:1092F000244B1A680723002A06D01668002E03D0D4
:10930000290001AAB04703006A4613706B461B7818
:109310006088002B2AD1FFF767FC06B070BD1800EB
:1093200000F06CF9D4E7180000F087F9D0E71800D6
:1093300000F093F9CCE7180000F0ADF9C8E7180089
:1093400000F0C3F9C4E7180000F0F6F9C0E7180010
:1093500000F0F6F9BCE7180000F013FAB8E71800BF
:1093600000F013FAB4E707236A4613706946608871
:10937000FFF782FFD1E70523012AC5D1024BB8E7E9
:109380006164FF1FCC65FF1FD065FF1FF8B52C4F30
:109390008600F35904000D00002B40D0DA88824289
:1093A0003DD15A78062A33D11A78002A2ED00120CE
:1093B00099681A6A097D014206D0157B054203D0DF
:1093C00007225A700120F8BD0220014204D0157B0B
:1093D000054201D00922F4E70420014204D0127BA7
:1093E000024201D00B22ECE7164B1B68002BE9D0A0
:1093F0005B68002BE6D020009847BB5900215B78C2
:10940000122BDFD12000FFF715FFDBE70E4BECE757
:10941000112A04D1002900D032252900F2E7002DBD
:1094200008D12000FFF732F9002803D01023027979
:109430001343037121002800FDF798FAC2E7C046E4
:10944000D465FF1FCC65FF1FD065FF1F70B50E4EA2
:109450008500AB590400002B13D01B78002B11D1D1
:109460000A4B1B68002B04D05B68002B01D0200046
:10947000984773595B78122B03D100212000FFF726
:10948000D9FE70BD024BECE7D465FF1FD065FF1F0E
:10949000CC65FF1F094B8000C3581020002B0CD057
:1094A0001A6A002A09D09B68002B06D0127A1B7E0C
:1094B000101C9A4200D9181CC0B27047D465FF1F17
:1094C00070B503000D0014000220002A30D00029DE
:1094D0002ED013700B78081D53704B789370FFF7E4
:1094E000A7FCE070012002212B7A23716B7B0340E3
:1094F00063716A7B0A401343042263716E7B1640DA
:10950000334363716E7BF608F600334363712B7B44
:109510000340A371287B014000200B43A371297BEA
:109520000A401343A3712A7BD208D2001343A371CC
:1095300070BD10B50A0001000120FFF7C1FF10BD8A
:1095400010B50A0001000220FFF7BAFF10BD70B588
:1095500006000C000220002E30D000292ED0737897
:10956000201D0B70B3784B70F178FFF76DFC012272
:109570003579257271794B100800134093401040E3
:109580000343881010408000C9080343C9000B43FF
:109590006373B1794B1008001340934010400343AC
:1095A000881002409200C9081343C9000B432120D0
:1095B0002373FCF773FE854201D2122070BD222076
:1095C000257AFCF76BFE8542F7D823781820042B08
:1095D000F4D86378012BF1D80020EFE7030010B531
:1095E0000220002909D0002B07D00322481C0A7052
:1095F00019000D3202F068F8002010BD03000222AD
:10960000080010B5002B06D0002904D00E32591CDA
:1096100002F05AF80022100010BD030010B502201D
:10962000002909D0002B07D00422481C0A70190019
:109630000C3202F049F8002010BD10B5FFF7DEFF34
:1096400010BD03000220002906D0002B04D0052203
:1096500000200A701B784B70704703000220002B1B
:1096600008D0002906D05B7800200B70013B082B46
:1096700000D918307047030010B50220002909D026
:10968000002B07D00622481C0A7019000A3202F08B
:109690001BF8002010BD10B5FFF7B0FF10BD020091
:1096A0000B00022010B500290ED0002A0CD0072193
:1096B0001970118859701188090A997011180822B7
:1096C000D81C02F001F8002010BD03000A0002209F
:1096D00010B5002B0CD000290AD0997858780902CF
:1096E00001431180901CD91C082201F0EDFF0020DD
:1096F00010BD030010B50220002909D0002B07D0AF
:109700000822481C0A701900921801F0DDFF0020A1
:1097100010BD02000B00022010B500290BD0002A5A
:1097200009D009211970117818185970511C062296
:1097300001F0CAFF002010BD10B5FFF75FFF10BD9C
:1097400002000B00022010B5002A09D0002907D022
:109750005178197011180622581C01F0B5FF00202D
:1097600010BD030010B50220002909D0002B07D03E
:109770000A22481C0A701900063201F0A5FF0020D9
:1097800010BD10B5FFF73AFF10BD02000B0002201C
:1097900010B5002A06D0002904D018005178FFF730
:1097A00053FB002010BDF0B585B017001E006A46BF
:1097B00006230500080091819380FEF7C0FC132466
:1097C000011E02900CD03800B047041E05D12800BD
:1097D00001A9FEF76FFA041E02D0029801F08CFF77
:1097E0002800FFF701FA200005B0F0BDF0B5040035
:1097F0008BB0019115000021102202A801F0B4FFE6
:10980000334EA700B85900283CD0C388A34239D1B1
:109810000378002B36D14278062A18D102000100C5
:10982000553235310C3006ABFFF7A9FA002829D1A3
:109830002000FFF72FFE020006A902A801F044FF56
:10984000200002A901F058FE01200BB0F0BD816E8E
:10985000002917D00B8A112A28D19D420ED10198D8
:109860001231093A01F0A0FD012807D1BB592000AF
:109870009D6EFFF70FFE29000200DEE73221200077
:10988000FFF7D8FC2000FEF701FF061E1BD0416A3F
:10989000002918D00B8AAB4215D108220198123149
:1098A00001F082FD01280ED1716A0AE09D42E9D1E2
:1098B00008220198123101F077FD0128E2D1BB594D
:1098C000996E8A7EB9E7200001F0AEFDBCE7C04684
:1098D000D465FF1FF0B56B4D87007E5985B0337896
:1098E00002900393002B00D087E0B368346A0193A1
:1098F0007078062817D101221B7D134202D0217BEC
:10990000114218D10222134202D0217B114251D1BF
:109910000422134203D0237B134200D08BE0019B2F
:109920005A7DEB5991E007380428F8D801F064FF1C
:10993000032E42678300B36E002B03D11C2001F07D
:10994000BBFDB066EB599C6E002C1CD01022002190
:10995000200001F009FF0298FFF79CFD01002000A4
:10996000FFF72DFA01F040FE20822000082112307E
:10997000FFF725FA0298FFF78DFDA076EB5921003D
:10998000D888FFF70FFC0822EB591CE0B36E002BC0
:1099900005D01A00198AF0881232FFF70DFC022256
:1099A000019B197DEB5911423DD0207B10423AD0EA
:1099B000073208E0F488FCF7DBFD01002000FFF728
:1099C00011FC0A22EB595A70029B9C002A595378C9
:1099D000073B042B11D8D088FEF758FE00284ED044
:1099E000C3895A08D2182849029B0298CB542B5994
:1099F00041180433254801F037FD05B0F0BDFCF7F0
:109A00009FFD03000120834201D100200393EB5905
:109A1000DE88FCF79BFD039902003000FFF7ECFBAA
:109A2000019AEB59117D042211420CD0217B114285
:109A300009D00B22C7E7F688FCF73CFD0100300097
:109A4000FFF7EEFB6BE7019A527D01210A4204D039
:109A5000607B084201D00C22B5E702210A4204D003
:109A6000607B084201D00E22ADE704210A4204D0F7
:109A7000627B0A4201D01022A5E71222A3E7FA2254
:109A80005200B0E7D465FF1FD865FF1F4B9E001141
:109A900010B5064B1A780423100018401A4200D063
:109AA0000348FFF727FA002010BDC0466164FF1F7E
:109AB0001443FF1F70B50400FFF7D4FA051E43D10D
:109AC0002000FFF77FFA234EA400A0598268937C00
:109AD000DB0708D50321036A1B790B40012B02D158
:109AE000017F0B430377431DD97F8B1E022B0DD8BB
:109AF000022900D00121C088FCF790FF04213359CE
:109B00001A7F59700A431A77280070BD01290CD1B9
:109B100002231022437000210C3001F025FE305941
:109B200010213530FFF74BF9EEE70529ECD1022380
:109B3000D118437010220C3001F0C6FD04233259B5
:109B4000117F0B431377EAE708251828DCD1053D80
:109B5000DAE7C046D465FF1FF0B58BB005914388A6
:109B60007E4F9E00F45915000493002C15D1012955
:109B700002D000200BB0F0BD101D57781678FFF70B
:109B800057F9EB68320002932B7A04990193009005
:109B90003B002000FCF70CFFEBE7E388049A9342BC
:109BA00001D00820E6E72378012B00D1D4E0059B03
:109BB000581E092800D9CFE001F01EFE05CE0A2963
:109BC000CC506C859AB229000498FFF773FFD1E757
:109BD000200029001022453001F076FDB9594B785C
:109BE000042B02D1013B4B70C3E70B000A00253365
:109BF00035320C310498FFF795F90498FFF702FA13
:109C00000522431E9841BB59C0005A70B2E720009C
:109C100029001022553001F057FD049B4F4C9D0048
:109C2000295904980A0006AB55320C31FFF77AF92E
:109C300029591022453106A801F0B6FB012808D1A8
:109C40000498FFF7F7F90590002804D106222B5954
:109C50005A7005988EE708230593FAE763780C2B72
:109C60007AD1E36E002B03D11C2001F025FCE066C5
:109C7000BB59D86E00286FD01022290001F024FDB6
:109C8000BB590498DC6EFFF705FC0D22A076BB598A
:109C90005A706EE7E06E00285ED063780D2B5BD1C2
:109CA0002B8808220382A91C123001F00DFDBB593C
:109CB0009A68517D0222114226D0186A407B1042D8
:109CC00022D00C32E4E763780E2B45D1236F002BB2
:109CD00003D1162001F0F0FB2067BB59186F002854
:109CE00003D01022290001F0EFFC0F22BB59CFE76F
:109CF00063780F2B30D1206F0622691C103001F0E1
:109D0000E3FCBB599A68517D0422114203D0196AC1
:109D1000497B1142D5D100210498FFF78BFA28E73F
:109D2000636F002B0DD0BB59586F0028F3D0102261
:109D3000290001F0C9FC0122BB5952425B6F1A6134
:109D4000E9E7142001F0B8FBBB5960675B6F002B9B
:109D5000E9D126E72978DFE707200BE7D465FF1F65
:109D600010B5064C207001F067FC06212078FDF745
:109D700091FF0348FEF778FC10BDC046E765FF1F62
:109D8000018F001100200BB270B50D00834216DA6E
:109D9000264B187801F0D8FD041E0DD00378922BC5
:109DA0000ED0A02B37D0224B1878FF283AD02100B4
:109DB00001F01AFB002835D180200002684070BDF8
:109DC00043780E2B0BD03E2BEDD18378052B12D090
:109DD000082BE8D181798088FFF7D8FA08E0154B85
:109DE00082889A42DFD183681878591CFEF7C0FE3A
:109DF000002817D1D7E7104B1B785B0712D50F4B04
:109E00001B68002B0ED09B68002B0BD0C289811DD4
:109E100080889847ECE7FFF741FAA068002801D056
:109E200001F06AFC200001F05FFCC5E7E765FF1F59
:109E30000D43FF1F182000006164FF1FD065FF1F46
:109E400010B50078FFF712FA10BD10B50078FFF7D3
:109E5000FDFA10BD0C234343084A10B59B185A68FD
:109E6000002A03D0012901D1904710BD9B68002B27
:109E7000FBD00029F9D19847F7E7C0460466FF1FD9
:109E800001238340094A10B5946B1C439463506BC3
:109E900098435063D46B20009843012901D12000DE
:109EA0001843D063116B0B43136310BD0080004057
:109EB000F0B500240127154B85B0DA6B144E0392E0
:109EC0001A6C0192DA64019BE3403B4217D0039D78
:109ED000E5403D400295E5B202992800FFF7BAFF40
:109EE000316A736A002908D03900002B01D0029929
:109EF00079402800FFF7C4FF01E0002BF9D10134BD
:109F00000C36172CDFD105B0F0BDC04600800040F4
:109F1000E865FF1F064B01215A68C2400A4204D07F
:109F20001B68C3401800084070471B6DF9E7C04626
:109F3000008000400122064B8240002903D0D968EE
:109F40000A43DA607047D9689143D960FAE7C0469E
:109F50000038004030B5032444430F4BE25C1B192A
:109F60009C785D7801232D1B0135AB40013BA3405C
:109F7000A140DB430C00122807D808499200521870
:109F8000116819402143116030BD054A11680B402A
:109F900023431360F8E7C046E7BB001108F0004018
:109FA00014F00040C21F70B5D4B20623092C0BD8A0
:109FB0000125084C9540002908D00021FFF7CAFF71
:109FC00023682B4323600023180070BD2368AB4334
:109FD000F8E7C04600380040214BF0B51B185B780D
:109FE000022B21D1032444431E4A1F4EA35C1219A5
:109FF0009478012215008540B76B013CE4B23D43E3
:10A00000A240B563194C122815D89B0000290CD129
:10A0100017495B1899680A439A600123205C154A26
:10A02000834011680B431360F0BD11495B189968B8
:10A0300091439960F1E70E4B00290DD159690A430C
:10A040005A61225C1328E8D00123203A93400A4940
:10A05000086803430B60E7E7596991435961F0E7EA
:10A06000E865FF1FE7BB0011008000402CBC001119
:10A0700000F00040A0F00040A4F00040F8B500243B
:10A080001B4E1C4D1C4B1B5D012B1FD1194A9269A5
:10A09000E2401A420BD00122B25693402200143AF9
:10A0A000D2B2022A09D815494A6913434B610134D7
:10A0B00002360C35172CE5D1F8BD0022B2560F49F7
:10A0C0009200521891680B439360F0E7022BEED197
:10A0D000E7B23800FFF71EFF01235840C1B2380035
:10A0E000FFF77AFF3800FFF715FF6877DFE7C04614
:10A0F000B9BB0011E865FF1FE965FF1F00F00040D4
:10A10000012202388240054B002903D059690A43D5
:10A110005A617047596991435961FAE70038004024
:10A12000F8B50E0001210F008740114A0400D368E2
:10A13000FD43BB43D360831E8B4201D8FFF7E0FF92
:10A1400000212000FFF72EFF0A4A0B4B5168012E19
:10A1500005D139431B1951605E700020F8BD2940BC
:10A16000516002221C1962709A6915409D61F4E7E2
:10A170000038004000800040E865FF1F012210B554
:10A180008240074B002906D019680A431A60012152
:10A19000FFF7C6FF10BD196891431960F7E7C04685
:10A1A000008000400C2370B5002543430A4A290073
:10A1B0009B181D70094B04001B185D70FFF7B0FF62
:10A1C0000123A340064928000A681A430A6005498A
:10A1D0000A689A430A6070BD0466FF1FE865FF1FA6
:10A1E000348000403080004070B504000E00FF282D
:10A1F00013D003250540FFF7D5FF084AA3089B00AD
:10A200009B183F22ED00AA40AE4019682000914300
:10A21000314319600121FFF78DFE70BD18380040F1
:10A22000F8B50C244443134B0500E4186368002B75
:10A2300003D1A3681220002B1AD0022201270E4B53
:10A2400000215B195A7028002770FFF769FF6368C7
:10A250001E1E08D0A3683E00002B04D02800FFF784
:10A2600059FE4640F6B228003100FFF709FE0020F3
:10A27000F8BDC0460466FF1FE865FF1FF7B5C420A0
:10A28000FF222B4B80001958002491433F3A0A4388
:10A290001A508022274F5202274E1A60274B1D5D0D
:10A2A000002D21D0A31E012B03D80121E0B2FFF71E
:10A2B00027FF012D18D11F4B9B69E3402B4213D080
:10A2C000E3B218000193FFF725FE01000198FFF7A4
:10A2D00055FFE3B2143B022B1DD801217156184AD9
:10A2E0008D405369AB4353613B7F002B0DD0E5B2EA
:10A2F0002800FFF795FF2800FFF70CFE7B7F010089
:10A30000834202D02800FFF7A5FD01340C37023646
:10A31000172CC3D1F7BD012100237156F3568D4090
:10A32000074A9B009B189A68AA439A60DCE7C046DC
:10A3300000E100E0E865FF1FB9BB0011E965FF1F00
:10A3400000F0004010B501210400FFF7E9FE0123F1
:10A35000044A002011194B70A34091690B4393618B
:10A3600010BDC046E865FF1F70B50E001500040063
:10A37000FFF718FF0C236343094A20009B189D60D8
:10A380005E60FFF74DFFF021064B074A8900051E6E
:10A390005A5002D02000FFF705FF280070BDC046CC
:10A3A0000466FF1F0000FF1FB19E001170B5134D22
:10A3B00007202C78002C1FD1982221005200280061
:10A3C00000F0EAFF0123C420FF222B700C4B800019
:10A3D0001C635C630B4B1C605C600B4B1958914316
:10A3E0003F3A0A431A50802252021A600D20074A4F
:10A3F000074901F049F8200070BDC046E865FF1F1D
:10A4000000800040A0F0004000E100E07DA20011CB
:10A410007DA00011030010B50620072B09D8054ABE
:10A42000137000F0D1FFD7210020034B034A8900AD
:10A430005A5010BD3C43FF1F0000FF1F8D1BFF1F24
:10A4400070B51D0002240C2910D8094ACA40D20751
:10A450000CD5FBF72FFF041E08D1059A049928009C
:10A46000FBF744FFFCF7B2FDFFF712FB200070BDC5
:10A470001210000030B50D7802232C009C431842C6
:10A4800001D02B431C0008252300AB43284201D0F8
:10A490002B00234320241D00A543204201D01C4350
:10A4A00025002A230D70184204D011781E3B0B435F
:10A4B000137030BD0028FCD10C2113788B43F7E7D3
:10A4C000F8B51D0006AB1B88140007AA0E000B2070
:10A4D0001778002B27D10A78022A49D14A68507888
:10A4E00011780002244A08438018042840D801F05B
:10A4F00083F903121D1B2300F06801F08DF8021C84
:10A50000C0B2B84200D93A1CD2B22000F1682A8009
:10A5100001F0DAF806E00222F3681B882A80237033
:10A520001B0A63700020F8BD0622EEE701232B8092
:10A53000F3681B782370F5E7F368002B16D0082228
:10A540002A801A8822701A88120A62705A88A270A9
:10A550005A88120AE2709A8822719A88120A6271E5
:10A56000DA88A271DB881B0AE371DBE72B80D9E76D
:10A5700001202B80D7E7C04600D6FFFFF7B51600B5
:10A580000A781D0008AB1F880C000123022A18D18D
:10A590004A685078117800022B4A08438018032833
:10A5A0000FD801F029F902254439E06801F034F8A8
:10A5B000C0B20723B84204D37B190193152B02DDE7
:10A5C0000D231800FEBDE0682A003100C01901F01B
:10A5D0007BF86B4600209B88E268D0541B4B1B68BD
:10A5E000834203D01B68834200D098470023E8E7EA
:10A5F0000B23002FE5D1022DE2D1737832781B02B4
:10A600001343E2681380114B1B68002BEED01B68CC
:10A61000002BEBD00120E8E70B23002FD1D1062D32
:10A62000CED12A003100E06801F04EF8DEE70B23BE
:10A63000002FC6D1012DC3D132787533012AC0D87D
:10A64000E3681A70D2E7C04600D6FFFFF467FF1F29
:10A6500070B50C001500072837D801F0CDF80414A8
:10A6600036361B36242E182015290BD8184E1622E4
:10A670000021300001F078F822002900300001F0BC
:10A6800023F8002070BD18200229FBD11288114B3D
:10A690001A80F6E718200829F4D10A000E4829008C
:10A6A00001F04AF9EDE718200129EBD10B4B1078A6
:10A6B0000B49DA69FFF7DEFEE3E718200129E1D153
:10A6C000064B10780749DA6BF4E70220DAE7C04658
:10A6D000DC67FF1FBA43FF1FB043FF1F4043FF1F4C
:10A6E0006843FF1F8843FF1F030010B50020DB07EE
:10A6F00004D50721024A034800F08CF810BDC0467B
:10A7000044BC00114043FF1F054A030010680028A5
:10A7100003D082889A4201D1806870470068F6E7CA
:10A72000EC69FF1F0A88030008009A4204D08A8857
:10A7300004309A4200D0002070470000F8B5F222A1
:10A7400000230D4F0D4E7968050042433370994246
:10A7500000D07B600A4C0021200001F005F80023A6
:10A760001A007C60AB4202D100203370F8BD013387
:10A770002280DBB2F234F5E7E46AFF1FE26AFF1FD2
:10A78000F069FF1F73B56B4601900600684615001F
:10A790001980FCF74DFF041E11D1002D0FD07689D2
:10A7A000002E11D00C2000F087FE00280ED0084AA1
:10A7B0000460136886808560002B02D11060200041
:10A7C00076BD1A001B68F7E70224F8E71324F6E7C2
:10A7D000EC69FF1F012100220A4B10B549420A4CC7
:10A7E000198099809A719A70084B20700120198005
:10A7F0005A60FFF7A3FF2078FCF778FF0448FDF7C5
:10A8000033FF10BDFC67FF1FEC6AFF1FE46AFF1FE8
:10A81000C1A80011022310B5002802D0FFF7B2FF33
:10A820000300180010BD0000030010B50020DB0776
:10A8300004D50421024A0348FFF7A4FF10BDC04617
:10A8400058BC0011C043FF1FF0B50E2687B003931C
:10A850000CAB1F8802ABF61805000800310002920D
:10A86000FDF768F804000120002C0FD03088FFF7B6
:10A870004BFF03000E20002B08D05E68002E05D091
:10A8800021002800039B029A0097B04707B0F0BD53
:10A890000A4B10B5984207D10122002352420A8088
:10A8A0008B708A808B7110BDFFF73CFF0028FAD0B7
:10A8B00001235B42038000238370F4E7FFFF000065
:10A8C000F8B5050001290AD1134E00243388F22778
:10A8D000AB4219D028001149FFF7DAFF06E0022940
:10A8E00004D10139FDF73EFF0028EDD0F8BD3B0053
:10A8F00063437268D018D35A002B09D03A00002164
:10A9000000F032FF0134E4B2054B1B78A342EED8CD
:10A9100001235B423380DDE7E46AFF1FFC67FF1F12
:10A92000E26AFF1F10B5FFF7FDFE0300002083421F
:10A9300000D0987810BD0000F0B589B01C000EABB7
:10A9400080CB03901E8810AB1B78049202930B7A85
:10A950000D00DB0616D42B780593022B24D0049827
:10A96000FFF7D2FE002812D003689C46002B0ED0C1
:10A97000029B2200019329003B0064460398009645
:10A98000A04705E00498FFF7BFFE002802D10E2083
:10A9900009B0F0BD8368002BF9D00A222900039882
:10A9A00098470028D7D0F3E76B6858781A786B4B34
:10A9B000000210439842D2D8043B984210D2684B10
:10A9C000984242D015D8674BC0180128C7D80B2031
:10A9D000002EDDD1EB681A7859683A80200028E013
:10A9E000614BC018032800D979E000F005FF846AA4
:10A9F000789E5E4B9842B2D10B20002EC8D1012325
:10AA00003B80EB6831001B7823706889013080B28D
:10AA1000FCF790FF3A88031E0ED0017802328A18A4
:10AA20003A80428962704289120AA270596802789B
:10AA3000E01C00F049FE06E004323A8031000422B6
:10AA4000601C00F091FE0020A2E70B20002E9FD199
:10AA5000EB6807A91E8804233B80330A3000267068
:10AA60006370FCF767FF051E28D004AB9A890E239C
:10AA700004A95B183E49C668FCF7D0FF00280BD13B
:10AA80002B783C486A680599FBF786FB002803D1C0
:10AA9000012304AA5B42D3813278022A06D171686D
:10AAA000201D00F011FE3B8802333B800E2304AAD8
:10AAB0009B181B88A3701B0AE370C4E704ABDE81FC
:10AAC000F4E70B20002E00D062E7E9680398FFF757
:10AAD00029FF02233B802070000A6070B3E70B203F
:10AAE000002E00D054E70222EB681B883A802370C6
:10AAF0001B0A6370A7E7E86800F08EFDC2B203008E
:10AB00000720B24200D243E70DD00299DBB27118A0
:10AB1000994202DB921BD3B20293029BE9681A00AE
:10AB20003B8089195AE70023F6E70B20002E00D05E
:10AB30002EE70722EB683A801A7822705A78627002
:10AB40005A88A2705A88120AE2701A792271DA8839
:10AB50006271DB881B0AA37175E7C04604290000F7
:10AB60000228000000D8FFFFFFD6FFFF03280000E7
:10AB7000FFFF000088BB0011F0B58DB06B460020D0
:10AB8000089120229B5E83423DDAA64B187800F0A4
:10AB9000DBFE071E32D00378B02B2CD100790238AF
:10ABA00016281FD800F048FE17001E001E001E00C9
:10ABB00031001E0096001E001D011E0052011E00E5
:10ABC00073011E00CD011E0050021E001E001E005B
:10ABD0008E021E00E302944B94491B8878880B80F8
:10ABE000FBF71AF83800FCF79BFF914B1B68002B12
:10ABF00001D038009847380000F076FD8020089B8F
:10AC00000002434018000DB0F0BDEE22002187483D
:10AC100000F0AAFD0BAA3B7B7989388900923A00A3
:10AC20000D32FCF79FFD0400804B1B78002C3FD1B8
:10AC300046E0804B788805937F4B4100CB5A0BAEA2
:10AC4000073BDBB232880293002301937B4B210048
:10AC500006930093059BFFF76FFE744D002810D1FB
:10AC6000069B3A8A1B889A420BD13800059912300C
:10AC700000F09AFB002804D02B7862899B00EB1827
:10AC80005A80162306A81B18328820007989FCF701
:10AC9000C5FE2B7804009A00AA1851880029C3D059
:10ACA0000133DBB22B70002807D006A9C98A918036
:10ACB000634A12889A42BCD802E00121494291803D
:10ACC000002B04D059497888FAF7DAFF8AE73E89E1
:10ACD0000A2479E000253E89574B06937B88069A23
:10ACE0005B009B5A033B9D4202DB002DF0D05BE0F2
:10ACF000162206A812183B7B798900923A00300090
:10AD00000D32FCF72FFD0590002858D04689017AB6
:10AD10007888FCF7F1FC041E44D1464B78880793F1
:10AD2000069B4100C95A454B0439C9B206AAD28ACA
:10AD300006930291019400930599079BFFF7FCFD90
:10AD4000041E2FD1069B39491A88931C002D26D149
:10AD50004B807988384B4900CB5A5119033B8B42C1
:10AD600020DD059B31485B8941190B71A91C013518
:10AD7000C9B2EDB2059145191B0A2B71059B2D49EE
:10AD80000433181800F0A0FC2C4B059A1B88D3182C
:10AD9000DDB22C4B9E4205D00136B6B29CE7498805
:10ADA0009942D6D0002D0CD0204C2800618800F0AC
:10ADB00023FB207021007888FAF772FF12E7059CC8
:10ADC000F0E7002C00D183E77B78142B00D109E752
:10ADD00016493B794E800B700C717888FAF712FF98
:10ADE00000E7162406ABE41821003889FCF7A2FD21
:10ADF000011E00D1B7E1788822880F4C45002C5BFA
:10AE00000A4D013CE4B2029400240F4B01940095DA
:10AE1000FFF792FD041E00D014E129007888FAF7AC
:10AE20004FFFDFE6EC6AFF1FAC42FF1F0468FF1F05
:10AE3000F867FF1FF868FF1F3464FF1FE869FF1FF2
:10AE4000AA42FF1FFFFF00000668FF1F162406AB83
:10AE5000E41821003889FCF76DFD011E00D182E164
:10AE600078882288AE4C45002C5BAE4D013CE4B2A4
:10AE700002947C89AC4B01940095FFF75DFD041EA4
:10AE800000D0DFE029007888FAF724FFAAE6002541
:10AE9000A44B1D803B00F6331B78A24A78880792AA
:10AEA000AB4208D99E4B12880693069943005B5A21
:10AEB000013B9A4203DB0799FAF716FF92E6162444
:10AEC0006B00FB18059306ABE418059B210018895D
:10AED000FCF730FD011E03D1059B01241E8973E799
:10AEE0007888924B2288069C099343001B5B904E06
:10AEF000013BDBB20293002300960193099BFFF70D
:10AF00001BFD041E02D0059B1E895DE77B88069A07
:10AF10005B009B5A079A108832881218934202DC11
:10AF20001B1A013B33807F4C02303288099900198B
:10AF300000F0CAFB2388328801359B182380EDB2CC
:10AF4000A8E70BAA3B7B7989388900923A000D3239
:10AF5000FCF708FC00250590059B002B04D10A2472
:10AF6000002D00D16EE060E0059B7888197AFCF72F
:10AF7000C3FB0100041E63D1694C6C4B78880694B6
:10AF80000993069B4400E45A694B063CE4B20BAEBD
:10AF9000328807930294019100930599099BFFF76A
:10AFA000CBFC041E4CD1079B5E491B881A1D002D4B
:10AFB00030D14A80059B5B4C5A8963191A716B1C0E
:10AFC0009BB2E318120A1A71162306A832881B18BE
:10AFD00079890598FCF722FDFF21AA1C2E1D033557
:10AFE0000B00059092B2B6B2ADB2002803D006AB0A
:10AFF000DB8AD9B21B0AA218651911712B714C4D4D
:10B00000301D2A884949201800F05EFB2B88F6186D
:10B01000B5B2A1E74988914207D17A8806995200D2
:10B02000525AEB18053A9A42C4DC3E4C280061881B
:10B0300000F022FC207021007888FAF75FFED1E54D
:10B04000002DF2D13E89BFE6162606ABF618310078
:10B050003889FCF76FFC3D000400FA3500282DD03C
:10B06000037A9B060CD400227B8939897888009268
:10B070003A000C32FFF7E8FB041E10D03E8915E0C1
:10B080003088FFF741FB00281AD08368002B17D0C7
:10B090002100122278889847041EE4D0EEE72B782E
:10B0A000002B02D17888FAF739FE00262B78002B86
:10B0B00000D097E5002C00D194E585E60124DDE77A
:10B0C0000E24DBE7162506ABED1829003889FCF7BE
:10B0D00031FC041E47D0037A9B0611D4154A7B88A5
:10B0E0001188994203D01448814207D11380134B31
:10B0F000F2261D780023D9B2A94221D30924A1E761
:10B100002888FFF701FB00282FD08368002B2CD064
:10B110002100122278889847041EDFD092E7C046AB
:10B120003464FF1F0468FF1F0668FF1FF868FF1FD5
:10B13000E869FF1FE46AFF1FFFFF0000E26AFF1FCC
:10B1400031005943546801336018615A0029D2D143
:10B150003C0008342100F22200F0B6FA2100788881
:10B16000FAF7E4FD3EE501246CE70E246AE71D4B87
:10B170001A887B889A4231D07888FAF7E1FD31E568
:10B18000F223059851684343CD18C95A00291FD0AE
:10B190003B7A012B0BD16C88AB887888AA1D009470
:10B1A000FFF752FB041E02D000233B722E88F222CE
:10B1B0000021280000F0D8FA00232B80059B0133E2
:10B1C000DBB20593084B05991B78064A8B42D7D80A
:10B1D00001235B421380002CCED0F5E5002634001D
:10B1E0000596EFE7E46AFF1FE26AFF1F70B50400EF
:10B1F0000E001500FFF796FA031E08D1310005482E
:10B20000FFF790FA03001120002B02D01C800020D1
:10B210009D7070BDFFFF0000F8B50B4F06003B7836
:10B220000D001400FF2B0ED00A2000F04DFB011E74
:10B2300009D0B1230380002346800371C5800481B7
:10B24000387800F0D1F8F8BD0144FF1FF7B50F00C2
:10B2500008A90600088809A90B240988002821D11B
:10B260000234022B1ED1557813782D021D432B007A
:10B270008B4301937334002B14D1FB683000190009
:10B280000093FFF74FFB019C85420BD02A00300052
:10B290000099FFF7ABFF041E04D12A003000798922
:10B2A000FFF7BAFF2000FEBDF0B50E7885B0039021
:10B2B0000AA805880120022E0DD14C6827786478F1
:10B2C00024023C43054FBC4205D10398DBB20196F2
:10B2D0000095FFF7BBFF05B0F0BDC0460229000096
:10B2E000034B10B51B68002B00D09847FEE7C04603
:10B2F000F06AFF1F07B501A8FFF7F2FF044A0548EF
:10B300000021121A00F048F8F8F7B6FAFEE7C04636
:10B31000F46AFF1F0444FF1F01B40248844601BCC5
:10B32000604700BF3D36FF1F01B40248844601BCA0
:10B33000604700BF0D52010001B40248844601BCC1
:10B34000604700BF691F000001B40248844601BC89
:10B35000604700BFF938FF1F01B40248844601BCB2
:10B36000604700BF993AFF1F01B40248844601BC00
:10B37000604700BF6571010001B40248844601BC0A
:10B38000604700BF7918000001B40248844601BC40
:10B39000604700BFD91B000001B40248844601BCCD
:10B3A000604700BFB70E000001B40248844601BCEC
:10B3B000604700BFCD4C010001B40248844601BC87
:10B3C000604700BF5952010001B40248844601BCE5
:10B3D000604700BF8D1BFF1F01B40248844601BCBB
:10B3E000604700BFAD32FF1F01B40248844601BC74
:10B3F000604700BF594F010001B40248844601BCB8
:10B40000604700BF350E000001B40248844601BC0D
:10B41000604700BFC53AFF1F01B40248844601BC23
:10B42000604700BFE928000001B40248844601BC1F
:10B43000604700BF091B000001B40248844601BCFC
:10B44000604700BF3D18000001B40248844601BCBB
:10B45000604700BF2D2EFF1F01B40248844601BC87
:10B46000604700BF5147010001B40248844601BC57
:10B47000604700BFA946010001B40248844601BCF0
:10B48000604700BF4551010001B40248844601BC39
:10B49000604700BF0D31FF1F01B40248844601BC64
:10B4A000604700BF1D3AFF1F01B40248844601BC3B
:10B4B000604700BFED3AFF1F01B40248844601BC5B
:10B4C000604700BF3D4B010001B40248844601BC07
:10B4D000604700BFE548000001B40248844601BC53
:10B4E000604700BFC94A010001B40248844601BC5C
:10B4F000604700BF5D17000001B40248844601BCEC
:10B50000604700BF311B000001B40248844601BC03
:10B51000604700BF851F000001B40248844601BC9B
:10B52000604700BFA54F010001B40248844601BC3A
:10B53000604700BF8B52010001B40248844601BC41
:10B54000604700BFE538FF1F01B40248844601BCD4
:10B55000604700BFED4A010001B40248844601BCC7
:10B56000604700BF5549010001B40248844601BC50
:10B57000604700BF0534FF1F01B40248844601BC88
:10B58000604700BF056A000001B40248844601BC60
:10B59000604700BFB139FF1F01B40248844601BCB7
:10B5A000604700BF1147010001B40248844601BC56
:10B5B000604700BF2124000001B40248844601BC5A
:10B5C000604700BFC9A9000001B40248844601BC1D
:10B5D000604700BF291C000001B40248844601BC3A
:10B5E000604700BF8530FF1F01B40248844601BC9C
:10B5F000604700BF2951010001B40248844601BCE4
:10B60000604700BFDD66010001B40248844601BC0A
:10B61000604700BFB352010001B40248844601BC38
:10B62000604700BFDD52010001B40248844601BCFE
:10B63000604700BFC51D000001B40248844601BC3C
:10B64000604700BFC926000001B40248844601BC1F
:10B65000604700BF8D12000001B40248844601BC5F
:10B66000604700BF4550000001B40248844601BC59
:10B67000604700BFB54C010001B40248844601BCDC
:10B68000604700BFADAE000001B40248844601BC73
:10B69000604700BFC56D010001B40248844601BC8B
:10B6A000604700BF2526000001B40248844601BC63
:10B6B000604700BF6D30FF1F01B40248844601BCE3
:10B6C000604700BF3119FF1F01B40248844601BC26
:10B6D000604700BFE94C010001B40248844601BC48
:10B6E000604700BF9DA9000001B40248844601BC28
:10B6F000604700BF434D010001B40248844601BCCD
:10B70000604700BFD949010001B40248844601BC2A
:10B71000604700BF5522000001B40248844601BCC6
:10B72000604700BF0519FF1F01B40248844601BCF1
:10B73000604700BF456B010001B40248844601BC6C
:10B74000604700BFEDA5000001B40248844601BC7B
:10B75000604700BF4936FF1F01B40248844601BC60
:10B76000604700BF8552010001B40248844601BC15
:10B77000604700BF154D010001B40248844601BC7A
:10B78000604700BFF30E000001B40248844601BCCC
:10B79000604700BF1D4B010001B40248844601BC54
:10B7A000604700BF75A9000001B40248844601BC8F
:10B7B000604700BFE117000001B40248844601BCA5
:10B7C000604700BFD532FF1F01B40248844601BC68
:10B7D000604700BF3D37FF1F01B40248844601BCEB
:10B7E000604700BFF137FF1F01B40248844601BC27
:10B7F000604700BF090E000001B40248844601BC46
:10B80000604700BF1D3BFF1F01B40248844601BCD6
:10B81000604700BF2146010001B40248844601BCD4
:10B82000604700BF6DBC000001B40248844601BC03
:10B83000604700BF5125000001B40248844601BCA6
:10B84000604700BF313BFF1F01B40248844601BC82
:10B85000604700BF0124000001B40248844601BCD7
:10B86000604700BF055E000001B40248844601BC89
:10B87000604700BF156B010001B40248844601BC5B
:10B88000604700BF090E000001B40248844601BCB5
:10B89000604700BF7139FF1F01B40248844601BCF4
:10B8A000604700BF093BFF1F01B40248844601BC4A
:10B8B000604700BFF94C010001B40248844601BC56
:10B8C000604700BF3555000001B40248844601BC02
:10B8D000604700BF1D4D010001B40248844601BC11
:10B8E000604700BF6D36FF1F01B40248844601BCAB
:10B8F000604700BFB14E000001B40248844601BC5D
:10B90000604700BF4D1F000001B40248844601BCDF
:10B91000604700BF3139FF1F01B40248844601BCB3
:10B92000604700BF017F000001B40248844601BCAB
:10B93000604700BF014C010001B40248844601BCCD
:10B94000604700BF810E000001B40248844601BC7C
:10B95000604700BFF54E010001B40248844601BCB7
:08B96000604700BFC521000093
:10B9680000030103020003030402050206020700A4
:10B97800080309030A030B030C000D000E030F0351
:10B98800100311001303140315031603213C0011BF
:10B99800553C00110000000002000000AAB9001187
:10B9A800192A0F180A000000F1590000FD240000B0
:10B9B80041460100717D0011859D0011D97100116A
:10B9C800757B00118553001179AB0011E14F00110F
:10B9D800313E0011613F0011000000001616000002
:10B9E80002000000F4B90011F4FFF3FFD2FC0000DC
:10B9F800A1400011000000000000000054757961AA
:10BA08000042312E3900303031330067697468756F
:10BA1800622E636F6D2F707676780054484232003C
:10BA2800020000003CBA0011292A282A272A262ABF
:10BA3800252A242A0A180000E204000071020000E6
:10BA480078EC00000500000074400000102700009A
:10BA580060F000000400000006640000204E0000B2
:10BA680000000000060000005C44000010270000F1
:10BA78006CEE000007000000050000001F501D00CC
:10BA8800023CB4000001130019000000810200000C
:10BA980030313233343536373839414243444546FC
:10BAA8000000000089570011DD5700110000000058
:10BAB80002000000C4BA00116F2A6E2A1A1800008A
:10BAC80001A00000000000006410B71DC8206E3BF4
:10BAD800AC30D9269041DC76F4516B6B5861B24D8D
:10BAE8003C7105502083B8ED44930FF0E8A3D6D6F7
:10BAF8008CB361CBB0C2649BD4D2D38678E20AA05F
:10BB08001CF2BDBDFB349B5F80000080001000006C
:10BB180000000000DB5D001165740011FF5D00117D
:10BB28006D780011835E001143780011F95E0011F1
:10BB3800197800114B5F0011E1790011B35F001112
:10BB4800E1790011E55F00119B790011F95E0011A0
:10BB5800D1770011715F00117979001100000000A0
:10BB6800000000005760001179790011B9600011D8
:10BB78007D740011052A042A012A002A02290328B3
:10BB8800012800280118001800000000000000002B
:10BB9800000000000000008701010201020101020B
:10BBA800010203030401030101010101030302016E
:10BBB80003000D000E00100011001300140107010E
:10BBC80008010A010B011C011D02040205020702FB
:10BBD800080219021A021C021D03010302031700BE
:10BBE8000201000504000807000B0A001716001DD3
:10BBF8001C010201010504010E0D011110011413AD
:10BC0800011716011A19020201020B0A020E0D028F
:10BC18001110021413021716030504030807030B77
:10BC28000A030E0D0001020307090A0B0E0F10117B
:10BC380012141718191A1B1F20212200C1A4001161
:10BC48007DA5001100000000020000008EBB00115D
:10BC580000000000A9B2001100000000020000006E
:04BC68008CBB001180
:020000041FFFDC
:1000000000000000993D0011B0B90011ACB9001119
:100010003461FF1F0000000000000000000000002D
:1000200000000000000000000000000000000000D0
:1000300000000000000000000000000000000000C0
:1000400000000000000000000000000000000000B0
:1000500000000000000000000000000000000000A0
:100060000000000000000000000000000000000090
:100070000000000000000000000000000000000080
:100080000000000000000000000000000000000070
:100090000000000000000000000000000000000060
:1000A0000000000000000000000000000000000050
:1000B0000000000000000000000000000000000040
:1000C0000000000000000000000000000000000030
:1000D0000000000000000000000000000000000020
:1000E0000000000000000000000000000000000010
:1000F0000000000000000000000000000000000000
:1001000000000000000000000000000000000000EF
:1001100000000000000000000000000000000000DF
:1001200000000000000000000000000000000000CF
:1001300000000000000000000000000000000000BF
:1001400000000000000000000000000000000000AF
:10015000000000000000000000000000000000009F
:10016000000000000000000000000000000000008F
:10017000000000000000000000000000000000007F
:10018000000000000000000000000000000000006F
:10019000F932FF1F5931FF1FC16601000000000046
:1001A000000000000000000000000000000000004F
:1001B000000000000000000000000000000000003F
:1001C000000000000000000000000000000000002F
:1001D000000000000000000000000000000000001F
:1001E000000000000000000000000000000000000F
:1001F00000000000000000000000000000000000FF
:1002000000000000000000000000000000000000EE
:1002100000000000000000000000000000000000DE
:1002200000000000000000000000000000000000CE
:1002300000000000000000000000000000000000BE
:1002400000000000000000000000000000000000AE
:10025000000000000000000000000000000000009E
:10026000000000000000000000000000000000008E
:10027000000000000000000000000000000000007E
:10028000000000000000000000000000000000006E
:10029000000000000000000000000000000000005E
:1002A000000000000000000000000000000000004E
:1002B000000000000000000000000000000000003E
:1002C000000000000000000000000000000000002E
:1002D000000000000000000000000000000000001E
:1002E000000000000000000000000000000000000E
:1002F00000000000000000000000000000000000FE
:1003000000000000000000000000000000000000ED
:1003100000000000000000000000000000000000DD
:1003200000000000000000000000000000000000CD
:1003300000000000000000000000000000000000BD
:1003400000000000000000000000000000000000AD
:10035000000000000000000000000000000000009D
:10036000000000000000000000000000000000008D
:10037000F5B20011000000000000000000000000C5
:10038000000000000000000000000000000000006D
:10039000000000000000000000000000000000005D
:1003A0000000000000000000000000000D1BFF1F07
:1003B000000000000000000000000000000000003D
:1003C000000000000000000000000000000000002D
:1003D000000000000000000000000000000000001D
:1003E000000000000000000000000000000000000D
:1003F00000000000000000000000000000000000FD
:08183800006FFF1F4118FF1FA4
:10184000024981F3088802F09FF90000006FFF1F32
:1018500070B500241E491F4A1F484C6308CA1B0567
:101860001B0DE4188242F9D11C4B80228B630021AE
:1018700009201B4B920519621A4B1B4DDA671B4B53
:10188000DA688243DA609A68194802409A60112047
:10189000296002F08DF8112002F06AF880226B6C4A
:1018A000112093436B64EE23DB006343114A1B0C4E
:1018B00013840122104B9A7201F004FC0F4B1B7829
:1018C000002B04D10E4B1021187802F08DFB70BD57
:1018D000000005408805054000060540FF010000A6
:1018E00000F0004004E100E0003800403CF000401F
:1018F000FFDFFFFF0461FF1FB861FF1FE663FF1FEB
:10190000E461FF1F10B502F0B7F9072804D01228D0
:1019100008D0022808D010BD044A0420136B0133FC
:101920001363F8E70220F6E71420F4E7DC64FF1FF6
:10193000F8B507000C0026002500503630785135E8
:10194000002804D10300287058342370F8BD29788A
:10195000CA00481E8141A3183800A25C5B68C9B266
:10196000FFF7D0FF00280DD12B78DA00A218013341
:1019700050602B703378044A013B3370136A013393
:101980001362D8E70123DFE7DC64FF1F5C234343D6
:10199000074910B5C9180B0058331B78012B05D126
:1019A000FFF7C6FF034A936A0133936210BDC04636
:1019B0001065FF1FDC64FF1F10B502F09DF9064A99
:1019C0000121130010CB4942D967044B136002F088
:1019D000E3F8200010BDC04600E100E01000100058
:1019E00010B5040002F088F9024B1C6002F0D4F834
:1019F00010BDC04600E100E0431E5A425341A02200
:101A0000F0B5D2015B421340154D164A40019B18B8
:101A10002A18127E8BB00191002A1BD01A000832BE
:101A2000D46F0022E6B206AFE4B294420EDC28186E
:101A3000C369002B08D0019902AA117106AA049269
:101A400002AA167303A898470BB0F0BD1978B954D1
:101A50000132EAE71A7D1A7806AB01261A70E6E72A
:101A60009C67FF1F00400040F0B5254B040040017B
:101A7000C25C85B0002A2BD01A18117E002927D00D
:101A8000917E002924D01179022921D11689D78885
:101A9000D168F51BADB22A1C102D00D9102292B2CC
:101AA000BE4217D11818012303710023C269C380F5
:101AB00003819A4206D068460321037301710293A1
:101AC00001A890470820002C00D0192001F0FAFA54
:101AD00005B0F0BD013C65426C41A0256442ED01BA
:101AE0002C40084D1B186419074D0633013A92B279
:101AF000AA42EDD01888461C1E80085C2070F5E7CD
:101B00009C67FF1F00400040FFFF00000F220E4BAC
:101B100010B59868104002380A280BD801F0FEFF73
:101B20000D0A0B0A0A110A0A0A0A060002210020FD
:101B3000FFF762FF10BD0121F9E70020FFF794FFD6
:101B4000F8E7DB6FF6E7C046004000400F220E4B7F
:101B500010B59868104002380A280BD801F0DEFF53
:101B60000E0A0B0A0A120A0A0A0A060002210120BA
:101B7000FFF742FF10BD01210800F9E70120FFF740
:101B800073FFF7E7DB6FF5E70090004013B5334CC8
:101B90002378072B3DD8324B1A78324B002A39D1A3
:101BA0008022196852020A431A60252001F0C0FE03
:101BB00020232D4A11680B43802113606B460422B9
:101BC000C90508680733104228D080210422C905BE
:101BD000C86810422ED080212020C905CA688243DF
:101BE000CA6014221A701A78002A2FD18021C905E0
:101BF000C86820320243CA6014221A701A78002A78
:101C000028D11A4B1A7D22785A601D221A70593237
:101C1000DA6013BD1A6816490A40C5E7086802432E
:101C20000A6014221A701A78002ACED01A78013A63
:101C3000D2B2F7E7C8680243CA6014221A70197852
:101C40004A1ED2B21A700029F9D1C4E71A78013AB3
:101C5000D2B2C7E71A78013AD2B2CEE73C43FF1FAF
:101C60000444FF1F3CF000403443FF1F00200040AD
:101C7000FFFFFEFF564B70B51B68012B03D1554A81
:101C8000936D0133936502F0B7F9534B534A1860D3
:101C9000534B544C1A600123534A1360534A136048
:101CA0002378002B06D006225149524802F00CF846
:101CB00000232370504A514B10681B78C1B2002B8F
:101CC0000ED14F4CC0B223785BB2002B4FDB237890
:101CD00024785BB264B21B0424021B191B18136026
:101CE0000B1C50294ED95023464A47491078DBB285
:101CF000FF2202284BD10868444C454D267890437A
:101D00002A78964254D9227824782E78023B5D10A6
:101D1000A31B6B435201D31A10335B1118430860A5
:101D200002F04AF8031F012B45D83A4B1B78002BD1
:101D300006D0394B1B78002B02D0002002F0CCF8E3
:101D4000A122364B92009978354B4A431B689B1869
:101D5000832292009B181B78033B012B03D8AF20F2
:101D6000400002F051F801222E4BDA8270BD237838
:101D700024785BB264B2FF33FF341B0424021B19C6
:101D80000138ABE7CAB2022AAED20223ACE7086838
:101D9000254C264D267890432A78964208D92278F9
:101DA00024782D78023B5B10641B63435201B2E739
:101DB0002378DBB2B2E70228D5D11D4B1B78013B5B
:101DC000022B03D91B4B1B78022BCCD16C20C8E70C
:101DD0009809FF1FFC0FFF1F2864FF1FFF3F000033
:101DE000141003402C64FF1F0C100340001003402C
:101DF000D50BFF1F7211FF1FB40003408C09FF1F9A
:101E0000680AFF1F490AFF1F94000340460AFF1F8C
:101E1000470AFF1FF908FF1F2209FF1F300DFF1F90
:101E20003409FF1FBC0BFF1F440AFF1F450AFF1F99
:101E30001C09FF1F2309FF1F10B502F07DF80022C7
:101E4000014B1A8010BDC0462464FF1F10B502F07C
:101E500033F8A121054A89009478054A6143126844
:101E6000044B5218528C1A8010BDC046300DFF1F13
:101E70003409FF1F2464FF1F10B50D4B0D4A9978DC
:101E8000A1239B004B431268D218531DD97F0A4BE4
:101E90001B88994209D2441C07D0C82805D0D269B2
:101EA0005B1A5A43054B5343C01801F02DFF10BD78
:101EB000300DFF1F3409FF1F2464FF1F7102000053
:101EC00070B5244D2B68002B28D002F015F82B6834
:101ED000D8402B680400002B27D001F045FE2B686A
:101EE000D8401D4B1D4A9978A1239B004B43126893
:101EF000D118D25C91239B00002A20D0CA5801320D
:101F0000CA50174B17491B680868834214D3D23B49
:101F1000181A012A1AD0144B186070BD01F0ECFF9A
:101F2000124B196801F010FED3E701F01DFE0F4BB4
:101F3000196801F009FED4E70D495B18E8E7CA50BB
:101F40000C4B1B68DB68E418201AE4E7F530FF301F
:101F5000E1E7C0461C08FF1F300DFF1F3409FF1FBB
:101F60009C09FF1F2864FF1FA009FF1F1808FF1FFF
:101F70002DFF3F003064FF1F70B504000D002829BD
:101F800016D10300A433C2881B889B1A0B4A9BB24C
:101F900093420DD906006A3605223100653001F002
:101FA000DBFE002804D13100200001F025FF70BDC8
:101FB0002900200001F0F0FEF9E7C046FE7F000096
:101FC000F8B50500012001F08FFE134CA36AA26A48
:101FD0009342FBD1114E336002F01EF8104903000A
:101FE00008601048426894460F4A17680022BC45B2
:101FF00001D24268BA1A0D4802603268AD18A422B4
:10200000E562606A520302436262094A1278002A5A
:1020100001D00F3B0B60F8BD00F00040340AFF1FF9
:10202000E408FF1F28100040180AFF1F1C0AFF1FAA
:102030001C09FF1F70B580241025E405A3682B43FD
:10204000A36001F011FFA368AB43A36070BD000063
:10205000F7B5160080221C001023D205019191686B
:1020600005000B43936000225A4BD7301A6001F0F1
:102070004BFF9D232A002F009B00EB58CA32012101
:102080000092FC37002B01D00021009A386801F043
:10209000E3FD2900009BCB311A784F4BD3351A60F2
:1020A0004B780A781B0213438A7812041A43CB78C0
:1020B0001B061343494A1BBA13604B790A791B026A
:1020C00013438A7912041A43CB7931001B06134358
:1020D000434A1BBA13606B782A781B021343AA7811
:1020E00012041A43EB781B0613433E4A1BBA1360D3
:1020F000019A330213433C4A13603C4B22001B1BE2
:102100009C4603293DDCB3089A0013005142B21AE1
:10211000032A46D1354AE018511A827840781204D1
:1021200000020243E05C043302430A600022FF2BFA
:102130004BDDF0222E4B12011A600F222D4B1A603C
:102140002D4A1368002BFCD00023224A2749136034
:10215000091B321D0B191B68043A180A23706070A2
:10216000180C1B0EA070E3700434002AF2DC8022ED
:1021700010213B68D20501333B6093688B43936029
:10218000F7BD6346D578981893782D061B042B432A
:10219000157804392B43557804322D022B43036004
:1021A000AFE7022A0AD1114AE05C511AE2185278CC
:1021B000120202430A6004339BB2B7E7012AB5D189
:1021C0000A4A521AE15C1160F5E7084959180A6099
:1021D0000433ACE7000004403C00044038000440F5
:1021E00034000440300004400C000440000104406E
:1021F000040004401000044014000440F7B515002A
:1022000080221C001023D2050091916807000B4327
:1022100093600023654AD730136001F075FE9D235B
:102220003E009B00F9583B00CA363200FC330029BF
:1022300000D07FE0586801F00FFD390032785C4B28
:10224000CB311A604B780A781B0213438A78AC466C
:1022500012041A43CB78281D1B061343554A1BBA98
:1022600013604B790A791B0213438A7912041A43CB
:10227000CB791B061343504A1BBA13604B7A0A7A78
:102280001B0213438A7A12041A43CB7A21001B06DD
:1022900013434A4A1BBA1360009A2B021343484A5D
:1022A00013602200474B1B1B0093009BCE785B18EA
:1022B00001938B7836061B0433430E78043833437E
:1022C0004E78043136023343019E33600328ECDC40
:1022D0000321A808431C9B002940800003292BD11F
:1022E0003849E5185E18A9786D78E35C09042D0279
:1022F000294319433160030008330021FF2B2DDDF2
:10230000314B324919600F21314B196001232749A4
:102310000B60304B19680029FCD006211B680B406C
:10232000042B20D080220020D20593680A318B43F1
:102330009360FEBD01217DE7022908D121495D1886
:10234000E1184978E35C090219432960D3E70129C0
:10235000D3D11C495918E35C0B60CCE71948181815
:1023600001600433CAE7002310490B606346002B69
:102370000CDC3B00FC335A68102101325A60802289
:10238000D205936801208B439360D2E7009B9B1892
:102390001B68190A13705170190C1B0ED37004239B
:1023A0005B4291709C440432E0E7C0460000044068
:1023B0003C00044038000440340004403000044035
:1023C0000C0004400001044004000440080F000019
:1023D000100004401400044070B5061E19D00222FB
:1023E0005A4B9B799343012B13D1594B1A78FF2AEF
:1023F0000FD15A78FF2A0CD19A78FF2A09D1DA78BE
:10240000FF2A06D11A79FF2A03D15B79FF2B00D16D
:1024100099E0504B0C201A78012A08D000224E4D2A
:102420001A7029780B00093B042B01D8212070BDBC
:102430004B1F012BFAD9454CA37B042B00D982E01A
:10244000A279032A00D97EE09A1ED2B2012A02D8CC
:1024500060881F2877D9002E56D0012E73D1A0880E
:102460000128E3D0002907D1581E032803D801F022
:1024700055FB121715122E702978481E032811D803
:102480000025364B1D602823237501F00DFCA84262
:1024900027D0A580CAE702212970EDE70421FBE7D8
:1024A0000321F9E707390129C0D82D490968C96A0C
:1024B0008906BBD52B4908780028B7D1012A01D954
:1024C000002BB3D102230B708021274D26338901C5
:1024D0002878237501F000FC80212878890101F01B
:1024E00083FD0123A380214B1B78002B0AD0FA2205
:1024F00080211F4B92001B8809025A431A4B1878FF
:1025000001F08AFB002092E701F0F6FB2B78A68011
:10251000073B012B03D917482E7001F015FC114B16
:10252000114C1A78002A06D08021002220788901D7
:102530001A7001F0D1FB01F02FFB802120780902F5
:1025400001F0CAFBDEE7122071E7C046A60BFF1FB1
:102550006B09FF1F1A09FF1F1C09FF1F4809FF1FF6
:102560003064FF1F2309FF1F1B09FF1F2109FF1FE5
:102570002C09FF1F0010004010B5002901D001F008
:1025800043FB10BDF7B5604B01919978A1239B00E7
:102590004B435E4A060014681022E418D6235B0001
:1025A000E0583623FF33E35C00279343222B41D1CD
:1025B000574B0F3A1A600760012501F02DFC019B73
:1025C0001880E8235B00E35C002B01D0B34258DDA8
:1025D0000023504FFB70AD33FF33E3581A68002AD5
:1025E00003D09B88DB439B071DD03823FF33E35C7C
:1025F000002B18D09B235B00E35C002B13D1D1335D
:10260000FF33E35CB3420EDAA4235B00E15AE01827
:10261000090A023101F098FC23000122FE33013E39
:1026200001351A87FA70E8235B00E35C002B2AD09F
:10263000A8B2FEBD03683D00002BBED081880430E7
:10264000090A023101F080FCD6235B00E3581F60C9
:10265000B2E72300B133BA00FF33985801378188BD
:102660000430090A023101F06FFCE8235B00E35CEF
:10267000BB42EEDCE822F61AED1800235200A35408
:10268000A6E70027F1E7200001F0FEFB00281FD09D
:10269000002E1DDD7319882647190193B60020000E
:1026A00001F082FA5A308000201840680135818894
:1026B0000430090A023101F047FC200001F094FACD
:1026C000A3590133A351BD4202D0019B9D42E6D1E3
:1026D000114BE35C002BABD095239B00E35C002BFC
:1026E000A6D00E4BE15A0029A2D00D4AA35C994214
:1026F00002D90133A3549BE700231A212000A354DD
:1027000001F0CAFA94E7C046300DFF1F3409FF1FDD
:1027100000140340E010FF1F5A0200007202000084
:102720005E0200000D4970B54A6E0D4CD2038B69F4
:10273000D20BA24206D80B4D0224AA4204D901F0C2
:102740004BFA70BD02246442E21815007E24254035
:102750002242F4D0A3432B438B61F0E700F000400A
:102760000A200000FC1C0000F8B51D4B1D4F1A7814
:10277000002A10D1BA7B002A02D101321A7003E07C
:10278000032AFAD0022AF8D001F08EFA00220120A2
:10279000154B1A70F8BD154B154D1C68154B9E78DE
:1027A00001232B702878C0B200F09EFBBB7B002B6E
:1027B0000BD101F039FCA1239B007343E418832360
:1027C0009B00E41823782B70E4E7032B02D101F07F
:1027D000F3F9F0E70020022BDCD101F0A5FAEAE7DB
:1027E0001C09FF1FA60BFF1F2309FF1F3409FF1F32
:1027F000490AFF1F300DFF1FF0B587B00EAD2F78CF
:102800000FAD2D780593AC46634614000E4D0CAA0F
:1028100012782E7803930D9B009201932200059B62
:10282000029701F011FB2E70012C01D0042C08D16D
:10283000802206498B889343054A1278D2011343BC
:102840008B8007B0F0BDC0461C09FF1F6C11FF1F35
:102850007809FF1F0B001B3B70B504003020E02BF4
:102860000DD81300E025493BFF3B9BB2ED00AB4286
:1028700005D8034B200019825A8201F0DDFB70BDA0
:102880008410FF1F10B501F0B7FB054B00205B68FB
:10289000052B04D9034A5268D20200D4980810BD0F
:1028A00000100040FCE100E070B501F025FA0D4B8E
:1028B0001B68FC33DC691D6AFFF7E4FF641984427E
:1028C00004D2094B01241B68002B07D004220024EA
:1028D000064B1A70064A93690133936101F05CF963
:1028E000200070BD3064FF1F9809FF1F2309FF1FE0
:1028F000FC0FFF1F70B50C4D2B68FC335C6A01F0B8
:10290000FBF9FFF7BFFF2B680025FC339B6AE31838
:10291000834204D2054B1B68AB4200D1051B01F07A
:102920003BF9280070BDC0463064FF1F9809FF1FA7
:10293000D722044B92009B5810B5002B00D098472B
:1029400010BDC0460000FF1F10B501F0CFF8FFF723
:10295000EFFF2749274BCA6D274C1A4084235B00A1
:102960001343CB65254B1B68186A01F0BDF9244B56
:10297000244A1A60244B254A1A60A022244B520094
:102980001A60244B187801F04FF92000224901F019
:10299000F3F90023A3600233A360204B2049236096
:1029A00003232048A36001F0E7F910221E4BFF200B
:1029B0001A60802252031A60802292031A608022D9
:1029C00012041A6001F088FA012001F0D5F8FA200B
:1029D000400001F0F9F9582001F016FA134801F00F
:1029E000E3F9012001F0A8F9072001F0FDF910BD7D
:1029F00000F0004000FEFEFF141000403064FF1F96
:102A0000000003400180063DBC0003403408000084
:102A1000A40003404A0AFF1F71020000C30900001E
:102A2000FFFF3F002810004000E100E0307500008B
:102A3000674E336888331B6883F3088801F054FAC3
:102A4000644A6549136800200B401360634B644A75
:102A50001B68934200D1A6E001F086FA0221614A88
:102A600013688B431360FFF76FFF5F4B5F4C187861
:102A7000C0B201F0A9FA0023A3600233A3605C4B4B
:102A80000120236001F030F90323A36001F00CFA68
:102A9000040001F0B1FA050001F006FA554B186088
:102AA00001F0C2F9544B1968621A531EA14200D2B8
:102AB00013008022D203934201D39B029B0A326807
:102AC000D16AC90700D471E04C491C0C09689BB25B
:102AD0004C4359432402090A641803264849FC322E
:102AE00093680A6847489B1A474A0768126847492B
:102AF0009B18474A9A1833409208DB190A60036012
:102B0000042B03D9013233400A6003600E68414947
:102B1000A619300001F018F83F4F3E493B68C31832
:102B20003B603000019301F067F83C4E30680818B4
:102B300038493060884205D9019B01333B6001F080
:102B40005BF8316001F008FA354B1B78002B0DD093
:102B500001F052FA334B621B196812188A4232D2C2
:102B60004919091B091A304801F006F92F4E337A2A
:102B7000002B0ED001F040FA621BF168121891424E
:102B800024D94919091B091A294801F0F5F800232D
:102B90003372284B83F3088801F0C6F9002001F056
:102BA000E3F901F0E9F901F0DFF95CE7DC019900F4
:102BB0000234641A5900641A09214B438033CB4014
:102BC000A408E41889E7FA218900CCE71A49DBE771
:102BD0003064FF1F1CF00040FFFFC1FF0C0AFF1F05
:102BE000B641210310000040490AFF1F14100040A5
:102BF000C3090000100AFF1F340AFF1F380AFF1F15
:102C0000200AFF1F280AFF1F1C0AFF1F240AFF1F9C
:102C1000C4090000710200006008FF1F2C0AFF1F9A
:102C20001C09FF1FE408FF1F00100040740BFF1F6A
:102C30003C10004000000020DC050000A022054BF5
:102C400092009B5810B5002B01D0984710BD01F0A1
:102C50001BF8FBE70000FF1FA122054B92009B58C9
:102C600010B5002B01D0984710BD01F00DF8FBE71F
:102C70000000FF1FA222054B92009B5810B5002BAD
:102C800001D0984710BD00F0FFFFFBE70000FF1FD9
:102C9000A322054B92009B5810B5002B01D09847FA
:102CA00010BD00F0F1FFFBE70000FF1FA422054B61
:102CB00092009B5810B5002B01D0984710BD00F032
:102CC000E3FFFBE70000FF1F70B501F095F94F4BE4
:102CD000186000F041FF0400C30702D401F0ACF813
:102CE00070BD00224A4B1A604A4B187801380428FC
:102CF00029D800F013FF0320181C2400200000F046
:102D0000DBFF0128ECD0444C2378042B6ED101F07A
:102D10002BF80028E4D001F05FF8582001F074F897
:102D200002232370DCE7200001F0B6F8E9E7200079
:102D300000F082FFE5E7200001F08EF8E1E72000D7
:102D400001F02AF9DDE701F037F80500012808D184
:102D5000324B1B78053B012B03D82000FFF76EFF99
:102D6000D1E72D4B1B78022B01D0052B20D1022D52
:102D700028D12B4B9B7BAB431CD12000FFF76CFF72
:102D8000264B18780128BED16405BCD424492522DD
:102D90004B7B034205D1233A13405A425341263319
:102DA0001A000B7D9342AED9322001F0FDF8AAE75C
:102DB000022D07D1194B1B78052B11D12000FFF7ED
:102DC00059FFDDE7012D0BD1012B03D12000FFF7C7
:102DD0005FFF98E7062B03D12000FFF767FF92E71C
:102DE000200000F051FF022D8DD1C9E7032B04D143
:102DF0000C4B987C00F090FF72E7072B00D06FE738
:102E0000094B987B00F0E0FE6AE7C0469C09FF1F73
:102E10009809FF1F9009FF1F2309FF1F1C09FF1FAF
:102E2000A60BFF1FBC0BFF1FD40BFF1FFA210A4B81
:102E30000A4A49001A640A4A5A500A4A04395A503E
:102E4000094A08319A64094A5A50094A5C315A5071
:102E5000084ADA667047C0460000FF1FF927FF1FC7
:102E6000F528FF1FA928FF1FD923FF1F6927FF1F70
:102E7000791EFF1F4D1EFF1FF7B50B0CFF27012208
:102E8000009300233C001E001D009446019089B26F
:102E900062469A401000084018413618B6B2FF2F1B
:102EA00002D1012E00D19FB2009802401A41AD1804
:102EB000ADB2FF2C02D1012D00D19CB20133102BF9
:102EC000E6D10320012E07D1012D04D1019B24015D
:102ED000E4191C700138FEBD102EFCD10238102DF3
:102EE000F9D00230F7E700008023F7B59C46264B67
:102EF000264F01932649274A274D284C284B022864
:102F00001AD1604638600868264E30408026360365
:102F10003043086001990978002909D11660224AD6
:102F20002A60224A2260E02219689143A03A1BE0FD
:102F30008021C9021160F2E766463E600F68194EB3
:102F40003E408027FF023E430E6001990978002928
:102F50000DD1176001280ED1154A2A60154A22604A
:102F6000E02219689143C03A0A431A60F7BD8021F4
:102F700089021160EEE7E0210F4A02432A600F4AFE
:102F800022601A688A43F0E74B0AFF1FE000034003
:102F9000D80003409000034000000340500003406D
:102FA00040000340FFFFE3FF0280063D804508220A
:102FB0000180063D80660822008006988055082220
:102FC000F8B51E4B80261A680020140034403242A7
:102FD00032D11A681A4F32431A6001223B68063018
:102FE00093433B6000F080FE0122164D2B681E4388
:102FF0002E603B680A2613433B608027BF00124BBC
:103000001B683B4211D1013EF6B2FF2E09D17E2250
:103010000E4B1C682B68E40B1440934323432B6036
:1030200005E0082000F060FEE9E7002EEFD18022E5
:103030002B68600893432B60F8BDC046C4F0004085
:103040005CF0004018F0004068F0004060F0004084
:1030500010B500F0F9FD01215820034A00F0D4FF1B
:10306000FFF7AEFF10BDC046600AFF1F10B5782203
:103070000021034800F0B0FF00F0F6FD002010BD75
:103080002467FF1F70B5040000F036FE00230C20FB
:103090000B4A010059438D18515C00290DD0A14203
:1030A00008D1012300246B7000F086FF00F074FD4E
:1030B000200070BD01330A2BEBD11224F6E7C04685
:1030C0002467FF1F70B5040000F016FE00231900EE
:1030D0001D000D4A1078002806D0A0420CD1557072
:1030E00001310C320A29F5D1002B0AD100F0BCFDC8
:1030F00000F052FD002070BD5078461EB0411B18F4
:10310000EEE700F059FFF3E72467FF1FF7B504006F
:103110000C20002384460E4D019267465F43E85D14
:103120007E19A04212D000280BD10A4B9C46624661
:103130001B7808331370019B70707C557160B3600D
:10314000FEBD01330A2BE8D10320F9E70720F7E79A
:103150002467FF1F2067FF1F8020F8B5484BC0057C
:103160001B68C1248360474BFF251A680123134362
:103170004361454BA4001A68444B40211A60444BFC
:103180001A68444B1A60444B1A59AA431A51C52273
:1031900092009E58AE433143802699509F583F4934
:1031A000F6010F403E439E509E5880273602360A55
:1031B0003043985080201A5900020A4002431A51A5
:1031C00004341A59364E3F04324080263A431A518D
:1031D0001A5936061202120A32431A5108341A5981
:1031E00080260A4002431A51C32292009F58B446D7
:1031F000AF4337439F509F58294E0F4007439F507E
:103200009F58374080263604374380269F509F586A
:1032100036063F023F0A37439F50C0221F59AF4333
:103220003A431A511A591202120A1643C6221E5163
:1032300092009C58AC4365462C439C509C580025FA
:103240000C4020439850C72080001A58154C11405C
:10325000C02212020A431A50134B1B78DB08AB4200
:1032600001DC0020F8BD2378002B06D0A368002BDA
:1032700000D0984701350C34EEE71220F2E7C04643
:103280003843FF1F3443FF1FB0F000401C67FF1F8F
:10329000B4F000401867FF1F00E100E0FF00FFFFEF
:1032A000FFFF00FF2467FF1F2067FF1F030010B50B
:1032B0001F2809D8072200201340072404490A7850
:1032C000A24313430B7010BD00230620F5E7C04650
:1032D0002067FF1F054B06491B780A6805485B07F6
:1032E00002401B0B134300200B6070472067FF1F39
:1032F0001CF00040FFFFC1FF70B50C25FFF7EAFF8F
:103300000A4B1C780A4BE4086543ED18002C01D1E8
:10331000200070BD2B78002B06D06B68002B00D0EE
:103320009847013C0C3DF1E71220F2E72067FF1FB0
:103330001867FF1F1FB5002102220B0001910091A9
:10334000052000F021FD02230B490A681A42FCD136
:1033500020230393039B5A1E0392002BFAD1074AA2
:103360001368002BFCDA0B246C442000012100F0D0
:1033700083FD207804B010BD90C8004000C8004014
:1033800013B504000A4B0193019B002B01D11120BE
:1033900016BDFFF7CFFF23000340044205D00520F0
:1033A00000F0A2FC019B013BEDE71800F0E7C046EE
:1033B000FFFFFF0707B500F09FFC80220821D20520
:1033C000936A0191002B01D10739916202210C4AC5
:1033D00011600199481E01900029FAD10331116052
:1033E000053101910199481E01900029FAD111601F
:1033F000002B02D18022D205936200F0CDFB07BDE5
:1034000000C00040F0B52D4C89B02378002B4FD17F
:10341000FEF7D2FA02232A4F03903A681A42FCD1EF
:1034200020230693069B5A1E0692002BFAD1254EA6
:103430003368002BFCDA0120FFF7A2FF011E02D047
:10344000112009B0F0BD030003220190009005ADEA
:103450009F2000F099FC0321280000F00DFD0223BD
:103460003A681A42FCD120230793079B5A1E079201
:10347000002BFAD13368002BFCDA0120FFF780FF24
:103480000028DDD10398FEF7ABFAAA786B78110417
:103490001B020B4329780B4363601300113B0A495D
:1034A000052B07D801239340A3600B6001232370F1
:1034B0000020C6E780231B03F6E7C0462043FF1F1A
:1034C00090C8004000C800409808FF1F1E4B30B550
:1034D0005A6818781D4B85B0D31859424B410121C9
:1034E0000093002300F0F0FC194B1A4A02259A635E
:1034F00000221A6510325A658022C4219D65164B40
:103500001648D202DA6789004258154B80241A40C7
:1035100080231B0413434350642341200393E40599
:1035200000F006FA402000F003FA6562039D6B1E6E
:103530000393002DFAD103236362FFF73BFFA562DB
:10354000FFF760FF05B030BD2C43FF1F95FFFEF76E
:1035500000C80040050001FF04E100E000E100E0D8
:10356000FFFF00FFF0B585B00700FEF725FA022344
:1035700005002D4C22681A42FCD120230093009BA9
:103580005A1E0092002BFAD1284E3368002BFCDA29
:103590000120FFF7F5FE002803D01124200005B01C
:1035A000F0BD234B2360022322681A42FCD1202362
:1035B0000193019B5A1E0192002BFAD13368002B14
:1035C000FCDA0120FFF7DCFE0028E6D1194B1F6072
:1035D000022322681A42FCD120230293029B5A1E26
:1035E0000292002BFAD13368002BFCDA0120FFF79E
:1035F000C7FE0028D1D1104B2360022322681A4253
:10360000FCD120230393039B5A1E0392002BFAD173
:103610003368002BFCDA0120FFF7B2FE041EBCD198
:103620002800FEF7DDF9B9E790C8004000C8004067
:1036300001000006A8C800400180000110B500206C
:10364000FFF790FF10BD000010B5064B18705960D1
:10365000FFF73CFF00211320034AFFF757FD00202E
:1036600010BDC0462C43FF1FCD34FF1FF0B5040032
:1036700085B003920291FEF79FF9882263035B0BEA
:1036800052051A438023DB059D6A8023274F009251
:10369000BA68002601901B039A420CD9F823260031
:1036A0001B041E401C4206D08022214B52025E6247
:1036B00019680A431A60002D0BD100F01DFB02228D
:1036C0001C4B1A608023DB055A62013A9A6200F0B3
:1036D00063FA0023039A934220D1002D0AD100F00F
:1036E0000BFB144B03221D608023DB055A629D6295
:1036F00000F052FA8023BA681B039A4208D9002EC0
:1037000006D000220A4B0C495A621A680A401A6015
:103710000198FEF765F9002005B0F0BD009A029906
:10372000D2181278CA540133D4E7C0462043FF1F91
:1037300000C8004000C00040FFFFFEFFF0B587B0AA
:10374000029103920400FEF737F9019000F0D4FAD9
:10375000802302250122234EDB0535605D629A62DB
:1037600000F01AFA204F3B682B42FCD1202304932F
:10377000049B5A1E0492002BFAD11C4D2B68002B7F
:10378000FCDA0120FFF7FCFD002802D0112007B071
:10379000F0BD2000039A029900F0F6FB022304001A
:1037A0003A681A42FCD120230593059B5A1E0592C4
:1037B000002BFAD12B68002BFCDA0120FFF7E0FD8B
:1037C000051EE3D100F098FA80230322DB05356063
:1037D0005A629D6200F0E0F90198FEF701F9E0B24B
:1037E000D5E7C04600C0004090C8004000C8004077
:1037F000F0B5802489B00600FEF7DEF8E405A36A80
:1038000002250393029000F077FA0123304F3D60C8
:103810006562A36200F0C0F92E4C23682B42FCD1F4
:1038200020230593059B5A1E0592002BFAD12A4DA1
:103830002B68002BFCDA0120FFF7A2FD002803D043
:103840001124200009B0F0BD244B2360022322681C
:103850001A42FCD120230693069B5A1E0692002B87
:10386000FAD12B68002BFCDA0120FFF789FD021E3C
:10387000E6D11B4B03211E60030001900090202025
:1038800000F082FA022322681A42FCD12023079317
:10389000079B5A1E0792002BFAD12B68002BFCDAEB
:1038A0000320FFF76DFD041ECAD100F025FA802326
:1038B0000322DB053C605A629C6200F06DF9039BB9
:1038C000002B01D1FFF776FD0298FEF789F8B8E7E3
:1038D00000C0004090C8004000C800400100000641
:1038E00094C8004007B5000201910422000A01A912
:1038F000FFF724FF0EBD000073B5050005240B4A39
:10390000A3005B429B1819686B46DE1D3000FFF771
:10391000B3FA022804D133782B55013CEFD276BD9F
:10392000052CFCD00128FAD10230F8E71409001167
:103930001F2807D8012380228340D20591680B43BA
:10394000936070473F2808D80123802220388340A5
:10395000D20551690B435361F3E75F28F1D8012386
:10396000802240388340D205116A0B431362E8E796
:103970001F2807D8012280218240C9058B68934304
:103980008B6070473F2808D8012280212038824070
:10399000C9054B6993434B61F3E75F28F1D80122D6
:1039A000802140388240C9050B6A93430B62E8E7E7
:1039B0001F2810D880230200DB05153A1968012A58
:1039C00006D820229143196019680A431A6070478B
:1039D00001228240F6E73F2811D880230200DB0550
:1039E000353AD968032A06D810229143D960D9689C
:1039F0000A43DA60EBE7012220388240F5E75F28CE
:103A0000E5D842238022181A413B8340D205516AEF
:103A100099435162516A0B435362D8E710B50400D1
:103A2000012813D1A022184992050B685B015B099C
:103A300013430B60154B164A19681140154A0A4387
:103A40001A60402219680A431A6010BD0028FCD190
:103A500001000A2000F060FA21000B2000F05CFA5F
:103A6000C0220A4B920019680A4340211A601A6862
:103A70008A431A60B022044912060B685B015B0995
:103A800013430B60E1E7C04614F000401CF0004017
:103A90007F00FEFF80FD010072B6074A1368013304
:103AA00013600422054B1A600023054A136080222C
:103AB000D2055360FEE7C0467808FF1FC0F0004003
:103AC000C4F0004005490B68002B05D1044A0A6088
:103AD00004490A60044A13607047C046140AFF1F75
:103AE000841E0000380AFF1FC4F000400023034A70
:103AF0001360034A1360034A1360704754F0004098
:103B000040F1004044F1004002B4714649084900C8
:103B1000095649008E4402BC7047C04602B4714643
:103B200049084900095C49008E4402BC7047C04600
:103B300003B47146490840004900095A49008E44BF
:103B400003BC70470000000001B40248844601BC79
:103B5000604700BF090E000001B40248844601BC62
:103B6000604700BFBD0B010001B40248844601BCA0
:103B7000604700BF6D0B010001B40248844601BCE0
:103B8000604700BF6911010001B40248844601BCCE
:103B9000604700BFFDB2001101B40248844601BC79
:103BA000604700BF9DA9000001B40248844601BCE3
:103BB000604700BFD9B0000001B40248844601BC90
:103BC000604700BF75F8000001B40248844601BC9C
:103BD000604700BFC1F7000001B40248844601BC41
:103BE000604700BFD1AE000001B40248844601BC6A
:103BF000604700BF5976010001B40248844601BC09
:103C0000604700BF090E000001B40248844601BCB1
:103C1000604700BFE9D4000001B40248844601BCFB
:103C2000604700BF8B52010001B40248844601BCCA
:103C3000604700BFEDA5000001B40248844601BC06
:103C4000604700BF0534010001B40248844601BC4E
:103C5000604700BFED68010001B40248844601BC22
:103C6000604700BF2144000001B40248844601BC03
:103C7000604700BFADAE000001B40248844601BCFD
:103C8000604700BFE927000001B40248844601BC38
:103C9000604700BFE917010001B40248844601BC37
:103CA000604700BF53B9000001B40248844601BC1C
:103CB000604700BFA9D8000001B40248844601BC97
:103CC000604700BF0134010001B40248844601BCD2
:103CD000604700BFE94C010001B40248844601BCC2
:103CE000604700BFB352010001B40248844601BCE2
:103CF000604700BF0189000001B40248844601BC4E
:103D0000604700BF75A9000001B40248844601BCA9
:103D1000604700BF8937010001B40248844601BCF6
:103D2000604700BF4DF9000001B40248844601BC61
:103D3000604700BF19FA000001B40248844601BC84
:103D4000604700BFE512010001B40248844601BC8F
:103D5000604700BFC1A5000001B40248844601BC11
:103D6000604700BFCD4C010001B40248844601BC4D
:103D7000604700BF01D7000001B40248844601BC7F
:103D8000604700BF2D6C010001B40248844601BCAD
:103D9000604700BF496D010001B40248844601BC80
:103DA000604700BF51B8000001B40248844601BC1E
:103DB000604700BF8D11010001B40248844601BC78
:103DC000604700BFDD0C010001B40248844601BC1D
:103DD000604700BF8512010001B40248844601BC5F
:103DE000604700BF6DF6000001B40248844601BC84
:103DF000604700BFF90D010001B40248844601BCD0
:103E0000604700BF85C1000001B40248844601BC80
:103E1000604700BF7912010001B40248844601BC2A
:103E2000604700BFCD0C010001B40248844601BCCC
:103E3000604700BFC166010001B40248844601BC6E
:103E4000604700BFDD0A010001B40248844601BC9E
:103E5000604700BF9D6A000001B40248844601BC6F
:103E6000604700BFF535010001B40248844601BC3B
:103E7000604700BFDD3F000001B40248844601BC3A
:103E8000604700BF3D71010001B40248844601BC97
:103E9000604700BF71B0000001B40248844601BC15
:103EA000604700BF0934010001B40248844601BCE8
:103EB000604700BF156B010001B40248844601BC95
:103EC000604700BFF9ED000001B40248844601BC20
:103ED000604700BFC56D010001B40248844601BCC3
:103EE000604700BFED6B010001B40248844601BC8D
:103EF000604700BFC9A9000001B40248844601BC64
:103F0000604700BFE90B010001B40248844601BCD0
:103F1000604700BF8944000001B40248844601BCE8
:103F2000604700BF559F001101B40248844601BCA0
:103F3000604700BF7997000001B40248844601BC85
:103F4000604700BF8D82000001B40248844601BC76
:103F5000604700BFC115010001B40248844601BC9E
:103F6000604700BFD544010001B40248844601BC4B
:103F7000604700BF016C010001B40248844601BCE7
:103F8000604700BF8552010001B40248844601BC6D
:103F9000604700BF9573010001B40248844601BC2C
:103FA000604700BFF935010001B40248844601BCF6
:103FB000604700BF6137010001B40248844601BC7C
:103FC000604700BF21A9000001B40248844601BC3B
:103FD000604700BF8914010001B40248844601BC57
:103FE000604700BFB70E000001B40248844601BC20
:103FF000604700BF0D52010001B40248844601BC75
:10400000604700BFC95C010001B40248844601BC9E
:10401000604700BF0167010001B40248844601BC4B
:10402000604700BFBD5C010001B40248844601BC8A
:10403000604700BFE9F6000001B40248844601BCB5
:08404000604700BF116E000093
:10404800020000008ABB001101000000A0B90011A5
:104058000200000086BB0011010000008840FF1F1D
:1040680002000000A8B9001101000000B461FF1FA0
:104078000200000084BB0011030000002861FF1F3C
:1040880012000000020000008ABB001101000000BD
:10409800E8B900110200000086BB00110100000011
:1040A800E5B9001102000000F2B900110300000098
:1040B8006361FF1F0200000084BB001103000000C1
:1040C8007861FF1F0200000086BB0011010000009C
:1040D800E4B9001102000000F0B90011030000006B
:1040E8003961FF1F0200000084BB001103000000BB
:1040F8005A61FF1F020000008ABB00110100000086
:1041080028BA00110200000086BB0011010000005F
:10411800D141FF1F020000003ABA0011010000005F
:1041280023BA00110200000086BB00110100000044
:10413800D041FF1F0200000038BA00110100000042
:104148008061FF1F0200000086BB00110100000013
:10415800CF41FF1F0200000036BA00110100000025
:1041680013BA00110200000086BB00110100000014
:10417800CE41FF1F0200000034BA00110100000008
:104188000EBA00110200000086BB001101000000F9
:10419800CD41FF1F0200000032BA001101000000EB
:1041A80009BA00110200000086BB001101000000DE
:1041B800CC41FF1F0200000030BA001101000000CE
:1041C80004BA00110202020202020000000000000C
:1041D8000D0C0000054C0011C94B001198BA0011D4
:1041E80090011D0018001800FFFF070102030405D5
:1041F80006020106000000000000000000000000A8
:1042080000000000000000000000000000000000A6
:1042180003000000020000008ABB0011010000003A
:10422800B8BA00110200000086BB001101000000AE
:104238008C42FF1F02000000C2BA001101000000FA
:10424800AE61FF1F0200000084BB001103000000E4
:104258001864FF1F0200000086BB00110100000067
:104268008C42FF1F02000000C0BA001101000000CC
:10427800B061FF1F0200000084BB001103000000B2
:104288001064FF1F1200000000010000000001116F
:10429800FFFF0000504859360000000000000000F1
:1042A8000B000500F0000000B400002800280028DA
:1042B8003075A000A000A000A00000080008E001E0
:1042C800F000100010001000100010001000500046
:1042D8005000500010001000D0070000000000003F
:1042E8000F0001000500307507001000010081FF74
:1042F80000000000FF0000003D710011456F001133
:10430800D56C0011FFFF0100FF000000599B001150
:10431800D5980011ED970011000000000000000082
:1043280000000800040000003B0001085902E001F9
:1043380088212800FF000000020000008ABB00114D
:104348000100000050BC00110200000086BB0011F3
:1043580001000000BD43FF1F0200000082BB0011E6
:1043680001000000DC67FF1F0200000086BB00118F
:1043780001000000BC43FF1F0200000080BB0011C9
:1043880001000000BA43FF1F0200000086BB0011B5
:1043980001000000B843FF1F020000007EBB0011AF
:1043A80001000000B043FF1F180018001D00900115
:1043B8000200000302020000020000008ABB001194
:1043C8000100000064BC00110200000086BB00115F
:1043D800010000000044FF1F020000007CBB001128
:1043E80000000000000000000200000084BB001173
:0A43F80003000000FC67FF1F20FF18
:040000051FFF184180
:00000001FF
